:1000000002755C02782600000000000271C9000041
:1000100000000002788400000000003200000000B0
:10002000000000023E4200000000000272F70000E3
:1000300000000000000000000000000000000000C0
:100040005052343032207665722E3132382E322EB4
:1000500032204864773A482032392D30362D3035F9
:100060002032323A3037202075F00612011E22125B
:100070006E8D75F00612011E126E922212006F1222
:10008000006812006F12006812006F120068120000
:100090006F12006812006F75F01812011E22126EA6
:1000A0008D75F04B12011E126E922275510412389A
:1000B0000C123822126E8D75F0C812011E126E924B
:1000C0002275510512380C12382212009E75F01E4E
:1000D00012011E12009E2275510712380C1238228E
:1000E0001200882275510612380C12382212008E26
:1000F0002212007C12007C221200E41200E41200A2
:10010000E422C2A1C25812006F75F01212011ED271
:10011000A1C2582212006F75F01212011E22128223
:10012000EC201607C0F0123262D0F0D5F0F0227049
:1001300004A243B322C0E01412013ED0E022C0E08A
:10014000030303540F28F8D0E0C0E0540704F5F08F
:10015000E213D5F0FCD0E0227003D3802830E7030F
:10016000C3802223F9C3137004A243801814C0E093
:10017000030303540F2479F8D0E0540704F5F0E2A8
:1001800013D5F0FCE992E022C0E024B4F8E21201B9
:10019000584004D0E0C322D0E024CAF58274003471
:1001A00000F583E01201A82220E702C322C2E7C0C3
:1001B000E0C2E0700AA243B3D0E030E001B322B461
:1001C0007E03C380F3B40204A22380ECB40404A22F
:1001D0002480E5B40604A22580DEB40804A22B80A6
:1001E000D7B40A04A20A80D0B40C0AE5774578C3D4
:1001F0006001D380C3B40E0512714B80BBB41007ED
:10020000A25E725DB380B1B41206A25D822680A8A0
:10021000B41406A25DB026809FB41604A25E809836
:10022000B418077400127E59808EB41A0774011234
:100230007E598084B41C087402127E590201B8B43D
:100240001E087403127E590201B8B4200874041207
:100250007E590201B8B422087405127E590201B811
:10026000B424087406127E590201B8B42608740733
:10027000127E590201B8D0E0C3221243EEE56E604F
:1002800013B401051233388008B4020512334B80D1
:1002900000756E00123262E5795440600B20A808A8
:1002A000305505C25512337C127CAE22C2B612778D
:1002B000CF75380074031258E8E51E1258E8E51FA0
:1002C0001258E874571258E81202D5E5381258E867
:1002D0003099FDD3227885E6232354031258E87819
:1002E00086E630E402240A540F1258E87885E6C402
:1002F000540375F00AA4F5F0E6540F25F01258E8FF
:100300007884E6C4540375F00AA4F5F0E6540F258A
:10031000F01258E87883E6C4540775F00AA4F5F0A3
:10032000E6540F25F01258E87882E6C4540775F0B9
:100330000AA4F5F0E6540F25F01258E87886E60393
:10034000C454071258E822C0F075F0DCD5F005B2AD
:10035000B5126AC4C0F0120591D0F030E7EED0F0CB
:1003600022AAF0120347E5336530F5F0E534653134
:1003700045F0600C1204B8853033853134120347E0
:1003800012055612034712057E1203471204C58A4E
:10039000F022AAF0120347E5336530F5F0E5346545
:1003A0003145F0600C1204B88530338531341203C6
:1003B0004712054212034712057E1203471204C575
:1003C0008AF02279207530017531037532E0900092
:1003D000E01203471204B81203471205167900759C
:1003E0003001753104753200900100120347120488
:1003F000B812034712051679E0753001753105759D
:1004000032009002001203471204B812034712058B
:100410001685303385313422AAF0120347E533655F
:1004200030F5F0E534653145F0600C1204B88530E4
:10043000338531341203471204FE8AF022AAF012E7
:100440000347E5336530F5F0E534653145F0600C80
:100450001204B88530338531341203471204E68A1A
:10046000F022C0F075F00833C297928300D297D57E
:10047000F0F5D0F022C0F075F008C297D29700A234
:100480008233D5F0F5D0F022D2B7D297D283D28280
:10049000D28422E53133E5303322C3E5313322E51E
:1004A000322212046212049312046212049A120499
:1004B0006212049F12046222120488C284745312CE
:1004C00004A2D28422120488C28474581204A2D2D4
:1004D0008422120488C28474541204A2E4120462B6
:1004E000120475D28422120488C28474541204A2A5
:1004F000E4120462120475F608D9F9D284221204B7
:1005000088C28474541204A2E4120462120475F2C4
:1005100008D9F9D28422120488C28474541204A225
:10052000E4120462120475F0A3D9F9D284221204F1
:1005300088C0E0C28474841204A2D0E0120462D2A3
:100540008422120488C28474841204A2E612046213
:1005500008D9F9D28422120488C28474841204A2B5
:10056000E212046208D9F9D28422120488C2847487
:10057000841204A2E0120462A3D9F9D284221204E4
:1005800088C28474831204A2D2841282EC1282EC98
:1005900022C2847457120462120475D28422D28358
:1005A000D282D297D2B7D284B2B575F0021282EC61
:1005B000D5F0FAC2B7B2B575F0021282ECD5F0FAF6
:1005C000D2B7B2B5227530017531DB753200120336
:1005D000471208607533FF7534FF22AE83AD8290F9
:1005E000DB007F207404F97480F875300185833155
:1005F00085823212043D7880E66E702508E66D70C3
:100600002008E6601AB4FF028013167404F974809F
:10061000F8753001858331858232120392C322D36B
:1006200022A3A3A3A3DFBD80F490DB007F2074048A
:10063000F97480F875300185833185823212043D6A
:100640007880E66E700908E66D700408E6FC22A367
:10065000A3A3A3DF0A7CFF2290DB007F207BFF7433
:1006600004F97480F8753001858331858232120473
:100670003D7880E66E702C08E66D702708ECB4FFBC
:100680000D788076FF0876FF0876FF0874FFF67411
:1006900004F97480F8753001858331858232120344
:1006A00092C322BBFF107880E6B4FF0A08E6B4FFCD
:1006B00005C374209FFBA3A3A3A3DFA3BBFF02D3A7
:1006C00022EB232354FC2400F5827583DB500205C2
:1006D000837880EEF608EDF608ECF608E4F674048C
:1006E000F97480F875300185833185823212039266
:1006F000C32275830075F08E7530028583317532A3
:1007000000C0F0C083120347120860D0830583D075
:10071000F0D5F0E475830075F0DA75300385833128
:10072000753200C0F0C083120347120860D0830501
:1007300083D0F0D5F0E47533FF7534FF2275830064
:1007400075820075F08EC0F0C082C083753002855E
:1007500083317532001203471204B8D083D082C0AF
:1007600082C08375300085823175320012034712D2
:10077000057ED083D08205830582D0F0D5F0C77581
:10078000830075820075F0DAC0F0C082C0837530D6
:10079000038583317532001203471204B8D083D029
:1007A00082C082C0837530018582317532001203A8
:1007B0004712057ED083D08205830582D0F0D5F024
:1007C000C77533FF7534FF2275830075820075F09D
:1007D0008EC0F0C082C083753000858331753200D1
:1007E0001203471204B8D083D082C082C083753010
:1007F0000285823175320012034712057ED083D004
:100800008205830582D0F0D5F0C77583007582001C
:1008100075F0DAC0F0C082C0837530018583317510
:1008200032001203471204B8D083D082C082C08342
:1008300075300385823175320012034712057ED070
:1008400083D08205830582D0F0D5F0C77533FF755C
:1008500034FF22120488C28474501204A2D284226B
:10086000120488C28474811204A2D28422120488E1
:10087000C28474841204A2E8120462D9FAD28422D7
:10088000F8790012034712086DEAC0E085823085CE
:10089000833175320012034712057ED0E0FA0583DA
:1008A000DAE77533FF7534FF22120488C28474546A
:1008B0001204A2E4120462E4C0E0120475D0F02530
:1008C000F0D9F5D284227583007582028006758383
:1008D00000758200E475F08D858230858331753234
:1008E00000C082C083C0F0C0E01203471204B812F7
:1008F000034779001208A9D0F025F0D0F0D083D0BA
:10090000820583D5F0D2858230858331753200C06F
:10091000E01203471204B812034779201208A9D045
:10092000F025F07533FF7534FF227583007582035F
:100930008006758300758201E475F0DA8582308562
:100940008331753200C082C083C0F0C0E01203471B
:100950001204B812034779001208A9D0F025F0D08C
:10096000F0D083D0820583D5F0D27533FF7534FF84
:1009700005E02275830075F00075300085833175C0
:100980003200C0F0C083120347120860D083058391
:10099000D0F0D5F0E47533FF7534FF75830075F042
:1009A000DA753001858331753200C0F0C0831203DF
:1009B00047120860D0830583D0F0D5F0E47533FF8B
:1009C0007534FF2253590F53580F5318F053190F12
:1009D000C2AFE5582324B1F8E5184519F608A61A60
:1009E000055853580FE558B55905055953590FD2B5
:1009F000AFC3E55895595002241024F45003756391
:100A00000022E559B558057400780022C33324B19B
:100A1000F8E6C0E008E6F8D0E02253580F53590F2B
:100A2000C2AFE559B55804D2AFD322055953590F77
:100A3000D2AFC380F53008597885E6540FC0E0E6A0
:100A4000C4540375F00AA4D0F025F0FD7886E63092
:100A5000E402240A540FFE901A007F3C7404F974D7
:100A600000F87530018583318582321204187800D0
:100A7000E26D701708E26E701208E2C42354E0F5CC
:100A8000F07886E6541F45F0F68006A3A3A3A3DF03
:100A9000CB221277CF120A351277DEFEAFF07DFF40
:100AA0000DED30E70122D26575F004A424E0F58253
:100AB000E5F03400F583C082C0837880E0F6A308B7
:100AC000E0F6A308E0F6A308E0F6D083D0827880B1
:100AD00086830886827880B6FF0708B6FF03020B7C
:100AE00058C3E58233F582E58333F583E58224E05C
:100AF000F582E5833405F5837882E6705B08E6606D
:100B000057FB7402F97480F8753001858331858252
:100B10003212043DA3A37880E60856B4FF03020B0B
:100B200058788086F053F07F08E6C39EC5F09F405A
:100B30001E7025E5F06018BD001E20431B7880E67E
:100B4000A2E720E713E5F024FA400DD2748009787B
:100B500080E6A2E79265DBAABD00028028ED14C002
:100B6000E0030303540F2479F8D0E0540704FB7426
:100B700000D333DBFD306505FBE24B8004F4FBE280
:100B80005BF2020AA0B2651232AF406E20316B20D8
:100B9000170B204205306562800320655D30653BA0
:100BA00020423878B3E2702D20731F78B1E2602BB9
:100BB0001275186026F5F07518C0751909E5F0541E
:100BC0003F4400F51A1209C48005127518600C78AC
:100BD000B1E278B3F2D274D273801FC274C273A22E
:100BE000659242400D304312C24312335A1252876B
:100BF0008008204305D24312336D020AA01204621A
:100C000012049312046212049AD2E01204621204D3
:100C10009F12046222120488C2847454120BFDE4F1
:100C2000120462120475F608D9F9D28422120488DB
:100C3000C2847484120BFDE612046208D9F9D284CE
:100C40002290FC00753004753100753200C082C0FE
:100C500083754BFA1203471204B885306D85316CE9
:100C600079087880120347120C15120E3DD083D0FC
:100C7000827044C082C08378848683088682120C86
:100C8000EE402478828683088682120CEE40181289
:100C90000D0DE582600AE56AB56C0CE56BB56D0774
:100CA000D083D082020CC97882E6249AF6120E8094
:100CB000126783D083D0820531E53170020530A3FD
:100CC000E58245837087120CD07533FF7534FF229F
:100CD00078827600087600788476000876000876B8
:100CE00000087600756D04756C00120E5C22C082DF
:100CF000C083E5822400F582E5833480F5834005D6
:100D0000D083D08222D083D08290000022E58275E9
:100D1000F008A4F582E5F0C58375F008A42583F5F5
:100D200083E5F03404F56BE5822400F582E5833435
:100D300000F5835002056B85836A22126793D08386
:100D4000D08222C082C083120E1670EF7882868312
:100D5000088682120CEE40E3120D0D1210F7788017
:100D600076007884E518F608E519F6087600087626
:100D7000007408F97480F8856B3085833185823280
:100D80001203927404F97484F8856B30858331857D
:100D9000823212043D75F00478807984E66760023F
:100DA00080990809D5F0F5120E1D78828683088691
:100DB00082A3120CEE7882A68308A68278848683AA
:100DC000088682120CEE7882E66583700A08E66572
:100DD000827004A3120CEE7884A68308A682C06DEC
:100DE000C06C856B6D856A6C120E5CD0E0D0F0B57E
:100DF0006C09C5F0B56D028018C5F0C06DC06C857A
:100E0000F06DF56C7882E62499F6120E80D06CD0E5
:100E10006DD083D08222120E1D120E3D22856D30C0
:100E2000856C317532001203471204B87908788056
:100E3000120347120C15853033853134227885E64C
:100E400018261826182618245566700F7885E61877
:100E5000661866186618661864996622120E631280
:100E60000E80227885E6182618261826182455F6AE
:100E70007885E61866186618661866186499F6226A
:100E8000856D30856C317532001203471204B8123B
:100E9000034779087880120C2D12034712057E1241
:100EA00003471204C585303385313422120E167083
:100EB000307882E6C0E008E6C0E0088683088682D3
:100EC000C3D0E09582F582D0E09583F5835010453C
:100ED00082600CE5822400F582E5833480F583C3CB
:100EE00022900000D322C2B6120EACE433C0E075EB
:100EF000380074031258E8E51E1258E8E51F12582E
:100F0000E874531258E8D0E01258E874001258E818
:100F100074001258E8E5831258E8E5821258E8E5B3
:100F2000381258E83099FD22C2B6E5366004F4FF65
:100F30008004FF120CD075380074031258E8E51EC7
:100F40001258E8E51F1258E874561258E8EF125884
:100F5000E8E5381258E83099FD227401C0E0788045
:100F600075F008E4F608D5F0FBD0E0D322120EAC01
:100F700040E860E878848683088682120F80C32266
:100F8000C082C083E58275F008A4F582E5F0C583D0
:100F900075F008A42583F583E5F03404F56BE5824C
:100FA0002400F582E5833400F5835002056B740854
:100FB000F97480F8856B3085833185823212043D67
:100FC000D083D08222120EAC7F085005120CD07F45
:100FD000007882865A08865B08865C08865DC2B601
:100FE00075380074031258E8E51E1258E8E51F1220
:100FF00058E874541258E8E5361258E8EF1258E8E9
:10100000E536603CE55D655BF5F0E55C655A45F00D
:10101000600B855D82855C83120F808003120F5CFC
:10102000855D82855C83A3120CEE85825D85835C81
:10103000788075F008E61258E808D5F0F8D536C47F
:10104000E5381258E83099FDC322E5367007C2AF83
:10105000120EAC5005E536F4800C7884A65C08A628
:101060005D120E5CE536D2AFC0E0C2B675380074D2
:10107000031258E8E51E1258E8E51F1258E87455A7
:101080001258E8D0E01258E8E5381258E83099FDD7
:10109000D322C2B675380074031258E8E51E125800
:1010A000E8E51F1258E874581258E87420232354B6
:1010B000FC041258E874201258E890DB007F20747A
:1010C00004F97480F8753001858331858232120409
:1010D0003D7880E61258E808E61258E808E612580B
:1010E000E808E61258E808A3A3A3A3DFD2E5381264
:1010F00058E83099FDD3221277CF7886E630E402A3
:10110000240A540FC4F97885E6C4540375F00AA480
:10111000F5F0E6540F25F0C313497881F67885E69B
:1011200092E754C0F97883E6C4540775F00AA4F531
:10113000F0E6540F25F049F97884E6C4540375F0BD
:101140000AA4F5F0E6540F25F0F5F07882E6547025
:101150002345F07883F67882E9F622223044FD12A6
:101160006E8D75F00612011E126E9275F01412014A
:101170001EE540C2442285833085823175320012DB
:1011800003471204B87530037531DB753200120362
:101190004712057E7533FF7534FF22C082C0837508
:1011A00030037531DB7532001203471204B8D08367
:1011B000D082858330858231753200120347120553
:1011C0007E7533FF7534FF22745578807910F608E8
:1011D000D9FC7410F97480F88583308582317532BA
:1011E000001203927533FF7534FF7410F97480F8A0
:1011F00085833085823175320012043D7880791004
:10120000B6553B76AA08D9F87410F97480F885832E
:10121000308582317532001203927533FF7534FFC9
:101220007410F97480F8858330858231753200122C
:10123000043D78807910B6AA0508D9FAE422740131
:1012400022E422C0E0900000C082C083121176D058
:1012500083D082C082C0831211C8D083D08260073D
:10126000D0F043F001C0F0C082C08312119BD08344
:10127000D082A37400B583D07440B582CBD0E02275
:1012800078807910E6B5F0070805F0D9F7E4227404
:101290000122C0E078807910F60805E0D9FA7410D0
:1012A000F97480F87530037531DB753200120392E2
:1012B0007410F97480F87530037531DC75320012E2
:1012C00003927410F97480F87530037531DB753250
:1012D0000012043DD0F0C0F0121280701E7410F99C
:1012E0007480F87530037531DC75320012043DD01E
:1012F000F0C0F01212807003D0F022D0F022E51D71
:10130000C0E0121292D0F07006E5F0F412129222B0
:101310007564FF121470C2081209326001221203B0
:10132000C37401F97464F87530017531037532A026
:1013300012043D7410F97489F87530017531037524
:1013400032C01204187410F97499F87530017531AF
:10135000037532D01204187402F97466F8753001FE
:101360007531CE7532001204187416F974B4F8751C
:1013700030017531CE7532C012041878B49000CAAD
:1013800075F016E2F008A3D5F0F97416F974B4F804
:101390007530017531037532A11204187408F9749F
:1013A00000F87530017531D27532001204187800DA
:1013B0009002F375F008E2F008A3D5F0F9D208E442
:1013C00022798077E909E4A22692E0A22792E1A29D
:1013D0002892E2A22C92E3A24292E4F709A73909EB
:1013E000A73A09A73B7404F97480F8753002753187
:1013F0008E75320012039222D242D243C221C227FA
:10140000A227B392A5C222C228A228B392A6C22ABA
:10141000C22CA22CB39280227404F97480F8753027
:101420000275318E75320012043D7880B6E9C90824
:10143000E6A2E092269220B392A7A2E192279221FF
:10144000B392A5A2E292289222B392A6A2E3922A94
:10145000922CB39280A2E49242788076FF7401F9D4
:101460007480F875300275318E7532001203922245
:1014700078B475F016E4F208D5F0FB74FF78BCF28E
:1014800078BDF222E8C0E07861E2F572D0E0F8229F
:10149000E8C0E07862E2F572D0E0F822E8C0E078D7
:1014A00063E2F572D0E0F82275F00384B4010474AD
:1014B0001A8017B4020474228010B40304742A80C2
:1014C00009B4040474428002741A227403F9745E2D
:1014D000F875300075318C7532E5120418785EE2CB
:1014E0001214A87861F2785FE21214A87862F27898
:1014F00060E21214A87863F2785EE224FD9201E2C1
:1015000024E292027401F9745DF875300075318C33
:101510007532E2120418785DE224FD9204E224E2BE
:101520009205227403F9745EF875300075318C757C
:1015300032E51203617401F9745DF875300075319C
:101540008C7532E2120361227980774809774E095F
:1015500077800977A07404F97480F87530007531CC
:101560008D7532201203927404F97480F87530027C
:1015700075318D753220120392227404F97480F84B
:1015800075300075318D75322012043D7982E76423
:101590008022E4A21C92E0A21D92E1A21E92E2A28D
:1015A0002992E37980F77401F97480F87530007539
:1015B000318C7532E8120392227401F97480F87547
:1015C000300075318C7532E812043D7980E7A2E075
:1015D000921CA2E1921DA2E2921EA2E3922922791C
:1015E00080E4A22D92E0A22E92E1A22F92E2A21418
:1015F00092E392E492E5A23192E692E7F709E4A23F
:101600003092E0A23292E1A23392E2A23492E3A2BB
:101610003692E6A23792E7F709E4A23892E0A23ABE
:1016200092E2A23B92E3A23C92E4A23D92E5A23E6A
:1016300092E7F709E579F77404F97480F8753000DA
:1016400075318C7532EC1203927980E57AF4F709E2
:10165000E57BF4F709E57CF4F77403F97480F87519
:10166000300075318C7532E9120392227404F974DA
:1016700080F875300075318C7532EC12043D79803C
:10168000E7A2E0922DA2E1922EA2E2922FA2E39293
:1016900014A2E69231A2E709E7A2E09230A2E19219
:1016A00032A2E29233A2E39234A2E69236A2E79209
:1016B0003709E7A2E09238A2E2923AA2E3923BA273
:1016C000E4923CA2E5923DA2E6A2E7923E09E7F54C
:1016D000797403F97480F875300075318C7532E9CE
:1016E00012043D7980E7F4F57A09E7F4F57B09E720
:1016F000F4F57C227980F77401F97480F875300074
:1017000075318C7532E4120392227401F97480F8F9
:1017100075300075318C7532E412043D7980E72212
:101720007401F9744FF875300075318C7532FC1204
:101730000361227401F9744FF875300075318C75AE
:1017400032FC12041822784FE270067850F208F248
:101750002275F000303C0475F03CA4AAF075F00846
:10176000A4FBACF0EA75F008A42CFAC374FD9BFB53
:1017700074FF9A7850F2EB08F2227401F97452F86F
:1017800075300075318D753200120361227401F9D4
:101790007452F875300075318D75320012041822BC
:1017A0007402F9746FF875300075318C7532FD1262
:1017B00004187402F97471F875300075318D753242
:1017C00001120418227402F9746FF8753000753133
:1017D0008C7532FD1203617402F97471F875300072
:1017E00075318D753201120361227401F97455F857
:1017F00075300075318C7532F01203617401F97423
:1018000056F875300075318C7532F412036174012D
:10181000F97457F875300075318C7532F612036122
:101820007401F97458F875300075318C7532F21204
:101830000361227401F97455F875300075318C75A7
:1018400032F01204187401F97456F87530007531CD
:101850008C7532F41204187401F97457F87530005D
:1018600075318C7532F61204187401F97458F875D4
:10187000300075318C7532F2120418227401F9743B
:1018800039F875300075318C7532F8120392740195
:10189000F9743AF875300075318C7532FA1203928A
:1018A0007401F9743BF875300075318C7532FB1298
:1018B0000392227401F97439F875300075318C7512
:1018C00032F812043D7401F9743AF875300075313C
:1018D0008C7532FA12043D7401F9743BF8753000CE
:1018E00075318C7532FB12043D227402F9741EF8B6
:1018F00075300075318C7532E0120392227402F952
:10190000741EF875300075318C7532E012043D227A
:10191000E57C5402600375710378A17984AA718013
:10192000021819E7F5F066540F700E18E7C4F5F0C9
:1019300066540F7004DAEAE422E6540FC5F0540F3F
:10194000C395F092077401227885791F7A03E6C463
:10195000540FF309E6540FF30908DAF2791F78A45B
:101960007A06E6540FF6E36670080908DAF4E4C272
:101970004922792478A97A06C3E3961918DAFA92EB
:1019800007792478A97A06E3540FB40F08E6540FB8
:10199000B40F108008E6540FB40F0B80061819DA44
:1019A000E680CB740122C3E396B40902801214606E
:1019B0000FC3E3F5F0E695F0B4090280031470E379
:1019C000E9B41F04E4D249221918E366540F60F009
:1019D00080D1121948701D30491A203018751850DE
:1019E00085831985821A1209C47549B4757D00D2A0
:1019F00045D248E42204227408F97480F875300056
:101A000075318C7532C012043D0219107408F974D6
:101A100080F875300075318C7532C012043D121992
:101A2000D2227405F97480F875300075318C7532E6
:101A3000C0120392227403F97485F8753000753171
:101A40008C7532C512039222C082C083E5822420A5
:101A5000F582E583347DF5837401F9743CF87530C3
:101A60000085833185823212043DD083D082C082CA
:101A7000C083E58275F008A42420F582500205F0A9
:101A8000A8F0E58375F008A4282400F5837408F90C
:101A90007480F875300085833185823212043DD020
:101AA00083D082124D5322C082C083E58275F00834
:101AB000A42420F582500205F0A8F0E58375F00813
:101AC000A4282400F5837408F97498F8753000850B
:101AD000833185823212043DD083D08222C082C0FD
:101AE00083E58275F008A42420F582500205F0A851
:101AF000F0E58375F008A4282400F5837406F974D2
:101B000080F875300085833185823212043DD083A0
:101B1000D082227405F97480F87530007531007533
:101B2000322012043D021910900000121A481219B6
:101B300010223008F3751B00751C0075689F7569CD
:101B40000FE568251BC2E0F582E569351CF583C009
:101B500082C083E5822400F582E583341BF583741B
:101B600002F97480F8753001858331858232120460
:101B70003D78808683088682121A481219107005F3
:101B8000D0F0D0F022D083D082C3E58313F583E573
:101B90008213F582200714E58245836022E58224C2
:101BA000FFF568E58334FFF5698007A385821B850F
:101BB000831CC3E568951BE569951C40028082740F
:101BC00001223008397410F97480F87530017531CC
:101BD000CE75322012043D7898798075F00AE7B40A
:101BE000FF02801AB43C120809D5F0F2900FE87891
:101BF000C2E2F53C7854F2E42266540F60E97401C5
:101C000022900000121A481219D22278A4E6540F2A
:101C1000B40F03021CA520080280E6751B00751C8A
:101C20000075689F75690FE568251BC2E0F582E5C0
:101C300069351CF583C082C083E5822400F582E506
:101C400083343BF5837402F97480F8753001858321
:101C50003185823212043D78808683088682121A8A
:101C6000481219D27005D0F0D0F022D083D082C3B0
:101C7000E58313F583E58213F582200714E5824599
:101C8000836022E58224FFF568E58334FFF56980EF
:101C900007A385821B85831CC3E568951BE56995B1
:101CA0001C4002808274012278987A0579ACE6544F
:101CB0000FC4F5F008E6540F45F0F70809DAEF22F3
:101CC00075F01E1282ECD5F0FA1200E475F00F12D6
:101CD00082ECD5F0FA1200E475F00F1282ECD5F028
:101CE000FA1200E422120094B2B575F00F1282ECE1
:101CF000D5F0FA30B7EF22D216D2A3C256C2A2D282
:101D000059D2A1C258D2A4C257121CE5121CC0124B
:101D10001F5D12665F120CD01205C5C2A3C256C267
:101D2000A2C259C2A1C258D2A4C257126F0740051D
:101D3000C2AF0274D0120094B2B575F00F1282ECEB
:101D4000D5F0FA80E6C2A3C256C2A2C259C2A1C24D
:101D500058D2B775F0021282ECD5F0FA20B74412CF
:101D60006F0750028091D216D2A3C256C2A2D25996
:101D7000D2A1C258D2A4C257121CE5D2161266A52F
:101D8000401CC2A3C256C2A2C259C2A1C258D2A408
:101D9000C257121E8B12665F120CD01205C5C2AF5D
:101DA0000274D0126E92C01D1208CED0F0702CC3F7
:101DB000E51D95F0F57E121E1712157A6019D216E0
:101DC000900000121A48121E8B12665F120CD0127D
:101DD00005C5B2B5121E1712131022D2A3C256D2D5
:101DE000A2C259C2A1C258D2A4C257C216754BFA98
:101DF000C2A075F0641282ECD5F0FA126E8DD2A0FA
:101E000075F0641282ECD5F0FA126E92D2B712839A
:101E10000420B7C7021D5F1215B912166C12170AFB
:101E2000A2E0923FA2E19240A2E292411217331245
:101E3000178D1218331218B31217A07401F974B168
:101E4000F87530017531CE75323012041878B1E270
:101E5000B4FF02E4F27401F974B2F875300175311F
:101E6000CE75323112041878B2E2B4FF02E4F27493
:101E700004F974D1F87530017531CE75323212041F
:101E80003D1218FD1214CB12174622D216C2A3C25D
:101E900056C2A2C259C2A1C258D2A4C257C01EC0C3
:101EA0001F78809000007A08E6F008A3DAFA121F83
:101EB0005D78809000007A08E0F608A3DAFA9000D6
:101EC000001265CE121A22121A35D01FD01E121817
:101ED000EA22751E30751F30D21CC21DC21EC229D7
:101EE000C22DC22EC22FC214C231C230D232C2336E
:101EF000C234C236C237C238C23AC23BC23CC23D0B
:101F0000C23E757900757A00757B00757C00786F2C
:101F10007422F2087400F278717406F2087400F208
:101F2000C23FC240C241784F7404F278527409F241
:101F300078557401F278567402F278577404F27886
:101F4000587404F2753907753A00753B00740178CE
:101F50005DF2785EF2E408F208F2C2082212097318
:101F6000121ED21218EA1215921215DFC2E0A23F19
:101F700092E0A24092E1A24192E21216F4121720DE
:101F800012177A1217EA12187C1217C512152312AB
:101F90001548126F6122305B04C25B800975F00C3A
:101FA00020B205D5F0FAD322C322E8C0E0E9C0E0B0
:101FB000EAC0E0200437200134121F9650257551E5
:101FC00000785EE2600C75F0031282ECD5F0FA1234
:101FD0003531785DE2600C75F0031282ECD5F0FAD1
:101FE000123692D0E0FAD0E0F9D0E0F822200222B6
:101FF00020051F3069EDC082C083E570700812783B
:10200000F240031220291214841278C2D083D082A5
:1020100080D13069CEC082C083E570700312207F0A
:102020001279CBD083D08280BA30030C300409D22D
:1020300064C263785D0220413001F4D263C26478E7
:102040005EE2B40F028013B41007124EF5D2518035
:102050002D75F00384E5F0B40007124FD8D25180FB
:102060001DB40107124E70D2508013B40210124DED
:10207000E7400B784DE583F208E582F2D252223038
:10208000030C300509D264C263785D0220973002E8
:10209000F4D263C264785EE275F00384E5F0B400C4
:1020A0000912518B4020D251801CB401091251B346
:1020B0004014D25080101251B6400B784DE583F297
:1020C00008E582F2D25222D2538008C2531221393B
:1020D000753D00C215D25B754BFA74403016027420
:1020E0000CF548C251C244E5486039121FAA20517C
:1020F0003375F0031282ECD5F0FA12027A2016033F
:102100002015183044E120531B75486012115CB44F
:102110000B0D75F0081282ECD5F0FAD25180051241
:10212000212C80C3C250D2AF754BFA22533D07F821
:10213000E53D24A4C8F6053D2278A475F00874FF97
:10214000F608D5F0FB22305009201B03D21B22C217
:102150005022C21B22D2538004D25BC253C21575D7
:102160004BFAD21A7440301602740CF54812213919
:10217000753D00C251C250C244C252C25412027ACA
:1021800020160320152D121FAA2051292050262089
:10219000522330442D785DE27004C24480242053E1
:1021A0001475486012115CB40B1275F0081282ECC1
:1021B000D5F0FAD251757D03754BFA22757D031265
:1021C000212CE54860F23054FD80B0C0E012234875
:1021D000D0E04021302E0320431B205E18C0E012C7
:1021E0006E97126E85D0E0203A091282957518100C
:1021F0001209C4D322203A091282957518201209B7
:10220000C4C322D20B7518C0751900751A011209C2
:10221000C4302619205D1C20380DC2AF754CFF75E7
:102220004DF8D2AF126E7B7852E2F547222036038A
:102230001222D122E51A543F44C0F51A751908C27A
:102240005EC25D205C46126E71D25B803FE51A541F
:102250003F4480F51A751908D25E80E5E51A543FAF
:102260004440F51A751908D25DC25E205C1E126EDC
:1022700071D25B8017E51A543F4400F51A751908AE
:10228000D25DC25E8000205C03126E857518C0129C
:1022900009C42230150122C0E074108004C0E0742B
:1022A0001178A4760A0875F00A84F608A6F0753D40
:1022B00003D0E078ADF2087405F2D21522C20B7596
:1022C0004700C2477518C0751900751A021209C473
:1022D00022757D00D2457549B475185075190F7572
:1022E0001AFF1209C42275186075190F751AFF12AA
:1022F00009C4C245C2482275187075190F751AFFB6
:102300001209C422126F61E51A543F4400F51A7590
:10231000190B7518C01209C4227873F208F212382A
:10232000D67518C0751900751A501209C422400CD0
:10233000305C08C25C205D03126E7122205CFC12CE
:102340006E97126E85D25C2212267F400D122A3AB9
:102350004008122DF540031231B32212268A400D97
:10236000122A454008122E0040031231BE22A290CC
:10237000301C01B37859E233F22210760302272889
:10238000301608C37859E4F2022698E57B541060B1
:10239000033043EF7859E260EF0460030227262000
:1023A0001F0320234DD223300819C0E0C082C08310
:1023B0007400120188D083D082D0E0400302272627
:1023C0000223C37855E224B0401CC082C08390250C
:1023D000DDE225E00493F5F0E225E093D083D0829E
:1023E000C0F0C0E0E222E2751890751909F51A12E2
:1023F00009C4022726126BEF1200D70227267401A8
:1024000012220302272674011221CB40E80227265C
:10241000C2431222E6022726D270756F050223E717
:10242000C0E07401127E10D0E00223E720430320B5
:10243000370CC0E07404127E10D0E00223E70227BC
:1024400026743D02250A0223E7C0E0E57C540470AF
:1024500005D0E00223E7D0E0022726C0E0D37401D4
:1024600012232ED0E00223E70223E70223E77400C1
:102470001222930227267410122293022726741127
:102480001222930227267420122293022726740117
:10249000F97480F875300075318C7532F112043D95
:1024A0007880E61222930227267401F97480F87569
:1024B000300075318C7532F112043D7880E61222BD
:1024C0009D02272630741C78B2E2601778B3F2754B
:1024D00018C07519097401543F4480F51A1209C4D3
:1024E0000223F50227263074FAE478B3F27518C097
:1024F0007519097401543F4440F51A1209C40223A6
:10250000F5751A011223040223F5204308D2431261
:1025100022F70223F5C2431222E60223F5E579549D
:10252000106007E41223190223F5022726E57954E7
:1025300010600874FF1223190223F5022726751A6A
:1025400001122234022726751A011222750227264B
:10255000751A0112225C022726751A0112224D02F9
:1025600027267400127E1074011283380223F5743A
:1025700000127E3C74011283470223F57400127E20
:102580005940EC0225627402127E107401128356C7
:102590000223F57402127E3C74011283650223F556
:1025A0007402127E5940EC0225867403127E107468
:1025B000011283740223F57403127E3C74011283AA
:1025C000830223F57403127E5940EC0225AA30439E
:1025D000030225150227262043FA02250D2726236C
:1025E000FE2406241023E723E723E72418242024CD
:1025F0002C244123E724462449245B23E723E723B3
:10260000E723E723E723E723E723E723E723E7237A
:10261000E723E723E723E723E723E723E723E7236A
:10262000E723E723E723E723E723E723E723E7235A
:10263000E723E723E723E723E723E723E723E7234A
:10264000E72468246B246E2476247E2486248E243A
:10265000A924C424E62501250A251D252D253E256E
:1026600047255025592562256F257C2586259325EC
:10267000A025AA25B725C423E725CE25D723E778AB
:1026800055E2B40B03A22322C3222043097855E26A
:10269000B40D03A22322C322201F062023030227F6
:1026A00026C223300819C0E0C082C0837400120122
:1026B00088D083D082D0E040030227260226BF784C
:1026C00055E260DAB401061222BD022726B40203E5
:1026D000022726B40307D2431222F78049B409081F
:1026E000204336303733803EB40A02743DB40D0BBC
:1026F000E57C54047030740D022719B40E0BC374BA
:102700000112232E740E022719C0E024CED0E0500F
:1027100008C0E024B0D0E0500D7518A0751909F577
:102720001A1209C48000D27622A291301D01B3781A
:102730005AE233F222107603022AE3301608C378F5
:102740005AE4F2022A53E57B542060033043EF78C9
:102750005AE260EF046003022AE1201F0320244DA7
:10276000D224300819C0E0C082C0837401120188ED
:10277000D083D082D0E04003022AE102277E78563F
:10278000E224B0401CC082C083902998E225E00476
:1027900093F5F0E225E093D083D082C0F0C0E0E270
:1027A00022E275189075190AF51A1209C4022AE175
:1027B000126BEF1200D7022AE17402122203022ADE
:1027C000E174021221CB40E8022AE1C2431222E660
:1027D000022AE1D270756F050227A2C0E0740112CF
:1027E0007E10D0E00227A220430320370CC0E07403
:1027F00004127E10D0E00227A2022AE1743D0228D2
:10280000C50227A2C0E0E57C54047005D0E0022791
:10281000A2D0E0022AE1C0E0D3740212232ED0E05D
:102820000227A20227A20227A27400122293022AE0
:10283000E17410122293022AE17411122293022AE7
:10284000E17420122293022AE17401F97480F87570
:10285000300075318C7532F512043D7880E6122215
:1028600093022AE17401F97480F875300075318C97
:102870007532F512043D7880E612229D022AE1307D
:10288000741C78B2E2601778B3F27518C075190934
:102890007402543F4480F51A1209C40227B0022A78
:1028A000E13074FAE478B3F27518C075190974024E
:1028B000543F4440F51A1209C40227B0751A021297
:1028C00023040227B0204308D2431222F70227B084
:1028D000C2431222E60227B0E57954106007E412E1
:1028E00023190227B0022AE1E5795410600874FF29
:1028F0001223190227B0022AE1751A0212223402A9
:102900002AE1751A02122275022AE1751A021222B0
:102910005C022AE1751A0212224D022AE1740012A9
:102920007E1074021283380227B07400127E3C7449
:10293000021283470227B07400127E5940EC02292C
:102940001D7402127E1074021283560227B07402A4
:10295000127E3C74021283650227B07402127E5903
:1029600040EC0229417403127E1074021283740237
:1029700027B07403127E3C74021283830227B07462
:1029800003127E5940EC0229653043030228D0022D
:102990002AE12043FA0228C82AE127B927C127CB18
:1029A00027A227A227A227D327DB27E727FC27A2D6
:1029B00028012804281627A227A227A227A227A297
:1029C00027A227A227A227A227A227A227A227A2BF
:1029D00027A227A227A227A227A227A227A227A2AF
:1029E00027A227A227A227A227A227A227A227A29F
:1029F00027A227A227A227A227A227A22823282688
:102A0000282928312839284128492864287F28A1E5
:102A100028BC28C528D828E828F92902290B291418
:102A2000291D292A29372941294E295B296529721F
:102A3000297F27A22989299227A27856E2B40B037D
:102A4000A22422C3222043097856E2B40D03A22413
:102A500022C322201F06202403022AE1C2243008B8
:102A600019C0E0C082C0837401120188D083D08273
:102A7000D0E04003022AE1022A7A7856E260DAB412
:102A800001061222BD022AE1B40203022AE1B403C4
:102A900007D2431222F78049B40908204336303761
:102AA00033803EB40A02743DB40D0BE57C540470CF
:102AB00030740D022AD4B40E0BC3740212232E7488
:102AC0000E022AD4C0E024CED0E05008C0E024B0EA
:102AD000D0E0500D7518A075190AF51A1209C480B6
:102AE00000D27622A292301E01B3785BE233F2224A
:102AF000107603022E9E301608C3785BE4F2022E95
:102B00000EE57B544060033043EF785BE260EF04F6
:102B10006003022E9C201F0320254DD2253008196A
:102B2000C0E0C082C0837402120188D083D082D0FA
:102B3000E04003022E9C022B397857E224B0401C5F
:102B4000C082C083902D53E225E00493F5F0E22586
:102B5000E093D083D082C0F0C0E0E222E27518900A
:102B600075190CF51A1209C4022E9C126BEF120093
:102B7000D7022E9C7403122203022E9C740312218E
:102B8000CB40E8022E9CC2431222E6022E9CD27059
:102B9000756F05022B5DC0E07401127E10D0E0025B
:102BA0002B5D20430320370CC0E07404127E10D04C
:102BB000E0022B5D022E9C743D022C80022B5DC036
:102BC000E0E57C54047005D0E0022B5DD0E0022EDD
:102BD0009CC0E0D3740312232ED0E0022B5D022BA5
:102BE0005D022B5D7400122293022E9C741012223F
:102BF00093022E9C7411122293022E9C7420122296
:102C000093022E9C7401F97480F875300075318C34
:102C10007532F712043D7880E6122293022E9C74DE
:102C200001F97480F875300075318C7532F7120433
:102C30003D7880E612229D022E9C30741C78B2E210
:102C4000601778B3F27518C07519097403543F44BE
:102C500080F51A1209C4022B6B022E9C3074FAE420
:102C600078B3F27518C07519097403543F4440F5E0
:102C70001A1209C4022B6B751A03122304022B6B60
:102C8000204308D2431222F7022B6BC2431222E6E2
:102C9000022B6BE57954106007E4122319022B6BA9
:102CA000022E9CE5795410600874FF122319022B40
:102CB0006B022E9C751A03122234022E9C751A0385
:102CC000122275022E9C751A0312225C022E9C752C
:102CD0001A0312224D022E9C7400127E10740312ED
:102CE0008338022B6B7400127E3C740312834702FC
:102CF0002B6B7400127E5940EC022CD87402127EA9
:102D0000107403128356022B6B7402127E3C740300
:102D1000128365022B6B7402127E5940EC022CFC6C
:102D20007403127E107403128374022B6B740312EB
:102D30007E3C7403128383022B6B7403127E594012
:102D4000EC022D20304303022C8B022E9C2043FAF0
:102D5000022C832E9C2B742B7C2B862B5D2B5D2BC6
:102D60005D2B8E2B962BA22BB72B5D2BBC2BBF2B59
:102D7000D12B5D2B5D2B5D2B5D2B5D2B5D2B5D2B9F
:102D80005D2B5D2B5D2B5D2B5D2B5D2B5D2B5D2B03
:102D90005D2B5D2B5D2B5D2B5D2B5D2B5D2B5D2BF3
:102DA0005D2B5D2B5D2B5D2B5D2B5D2B5D2B5D2BE3
:102DB0005D2B5D2B5D2B5D2BDE2BE12BE42BEC2BB8
:102DC000F42BFC2C042C1F2C3A2C5C2C772C802C04
:102DD000932CA32CB42CBD2CC62CCF2CD82CE52C9A
:102DE000F22CFC2D092D162D202D2D2D3A2B5D2D8D
:102DF000442D4D2B5D7857E2B40B03A22522C3224C
:102E00002043097857E2B40D03A22522C322201FD4
:102E100006202503022E9CC225300819C0E0C0827E
:102E2000C0837402120188D083D082D0E0400302B4
:102E30002E9C022E357857E260DAB401061222BDCC
:102E4000022E9CB40203022E9CB40307D24312222A
:102E5000F78049B40908204336303733803EB40A3E
:102E600002743DB40D0BE57C54047030740D022ED9
:102E70008FB40E0BC3740312232E740E022E8FC058
:102E8000E024CED0E05008C0E024B0D0E0500D7572
:102E900018A075190CF51A1209C48000D27622A266
:102EA00085302901B3785CE233F2221076030232D6
:102EB00061301608C3785CE4F20231CCE57B5480C3
:102EC00060033043EF785CE260EF04600302325F3E
:102ED000201F03202B4DD22B300819C0E0C082C028
:102EE00083740A120188D083D082D0E0400302327A
:102EF0005F022EF47858E224B0401CC082C0839058
:102F00003111E225E00493F5F0E225E093D083D07F
:102F100082C0F0C0E0E222E275189075190DF51A32
:102F20001209C402325F126BEF1200D702325F74D3
:102F30000412220302325F74041221CB40E80232F1
:102F40005FC2431222E602325FD270756F05022F14
:102F500018C0E07401127E10D0E0022F1820430345
:102F600020370CC0E07404127E10D0E0022F18024B
:102F7000325F743D02303E02325F022F18C0E0E53E
:102F80007C54047005D0E0022F18D0E002325FC0FC
:102F9000E0D3740412232ED0E0022F18022F18025F
:102FA0002F18740012229302325F741012229302BF
:102FB000325F741112229302325F74201222930244
:102FC000325F7401F97480F875300075318C753298
:102FD000F312043D7880E612229302325F7401F905
:102FE0007480F875300075318C7532F312043D78B9
:102FF00080E612229D02325F30741C78B2E26017C4
:1030000078B3F27518C07519097404543F4480F5FB
:103010001A1209C4022F2602325F3074FAE478B320
:10302000F27518C07519097404543F4440F51A121A
:1030300009C4022F26751A04122304022F262043E6
:1030400008D2431222F7022F26C2431222E6022F91
:1030500026E57954106007E4122319022F26023264
:103060005FE5795410600874FF122319022F2602BD
:10307000325F751A0412223402325F751A0412226A
:103080007502325F751A0412225C02325F751A04EF
:1030900012224D02325F7400127E107404128338C3
:1030A000022F267400127E3C7404128347022F26DE
:1030B0007400127E5940EC0230967402127E107435
:1030C00004128356022F267402127E3C740412836B
:1030D00065022F267402127E5940EC0230BA740346
:1030E000127E107404128374022F267403127E3C25
:1030F0007404128383022F267403127E5940EC025B
:1031000030DE30430302304902325F2043FA02309E
:1031100041325F2F2F2F372F412F182F182F182FA5
:10312000492F512F5D2F722F182F772F7D2F8F2F23
:10313000182F182F182F182F182F182F182F182F57
:10314000182F182F182F182F182F182F182F182F47
:10315000182F182F182F182F182F182F182F182F37
:10316000182F182F182F182F182F182F182F182F27
:10317000182F182F182F9C2F9F2FA22FAA2FB22F56
:10318000BA2FC22FDD2FF8301A3035303E30513093
:10319000613072307B3084308D309630A330B03067
:1031A000BA30C730D430DE30EB30F82F183102316E
:1031B0000B2F187858E2B40B03A22B22C322204312
:1031C000097858E2B40D03A22B22C322201F062047
:1031D0002B0302325FC22B300819C0E0C082C083CB
:1031E000740A120188D083D082D0E0400302325F9B
:1031F0000231F37858E260DAB401061222BD0232DD
:103200005FB4020302325FB40307D2431222F78095
:103210004EB4090820433B3037388043B40A027467
:103220003DB40C028039B40D0BE57C54047030744D
:103230000D023252B40E0BC3740412232E740E020C
:103240003252C0E024CED0E05008C0E024B0D0E03C
:10325000500D7518A075190DF51A1209C48000D209
:103260007622E5795440601AE57A540270061223FA
:103270006E12237AE57A5404700612272912273534
:10328000800C12236E12237A122729122735122A54
:10329000E4122AF0122E9F122EABC21F204A0122E6
:1032A000C24A7518C0751900751A541209C422E86B
:1032B000C0E07855E2640360187856E26403601158
:1032C0007857E26403600A7858E264036003C380BD
:1032D00001D3D0E0F82212011430080C12685F40CC
:1032E0000390FFF11268A422C052123306D052227A
:1032F00030081312685F400390FFF11268A4500574
:10330000F5521268FB22E55270057552108023B405
:103310001005755211801BB411057552208013B42D
:1033200020057552FF800BB4FF05755200800375B0
:1033300052FF1269ABE55222C24375186075190F2E
:10334000751AFA1209C4C245C24822D243751870D0
:1033500075190F751AFA1209C422C24375186075DF
:10336000190F751AE01209C4C245C24822D243752A
:10337000187075190F751AE01209C422E4A226927A
:10338000E0A22792E1A22892E2A22C92E3F57475C2
:10339000750512384C740350041239D2221239AC1C
:1033A0007891E6C0E0E57A54026012D0E0C0E054C3
:1033B000071233DAD0E0C0E054071233DAE57A546A
:1033C000046014D0E0C0E0C454071233FFD0E0C062
:1033D000E0C454071233FFD0E022A223301C01B313
:1033E0004007D320E10A0233FEC320E2030233FE8A
:1033F000301C01B3E45001147859F212237A22A24E
:1034000024301D01B34007D320E10A023423C32036
:10341000E203023423301D01B3E4500114785AF260
:1034200012273522B40207205107C250C25202347B
:10343000B2C082C08390EA60E53D606324FB405FD8
:1034400078A4E6540F758300F582D53D028050754F
:10345000F00AA4F58275830008E6540F2582F582F0
:10346000D53D02803AE58275F00AA4F58285F083A5
:1034700008E62582F58250020583D53D028020E5CD
:103480008275F00AA4F582C0F0E58375F00AA4D035
:10349000F025F0F58308E62582F582500205837851
:1034A0004DE583F208E582F2C251C250D252D08378
:1034B000D08222C289C28BD293C2B422C0F075F0EE
:1034C000FAD5F0FD75F064D5F0FDD0F0221234BCD1
:1034D0001234BC1234BC1234BC1234BC1234BC22C0
:1034E000D293C2B475F00512830420B2061283048D
:1034F00030B203D5F0F112830422C0F075F008A2B7
:10350000E7B392B4C2931234BCC2B4D2931234BCA7
:10351000C0E0E430B201040030B201040030B20176
:1035200004D36003D5E001C3D0E033D5F0D1D0F0AF
:1035300022D293C2B4D2B21234BCC2931234CDD2CE
:10354000931234CD20160330641C789076010874F1
:1035500080F608A2A3B392E4F6749008F608F60881
:10356000F608F60235A6789076030876800874800F
:10357000A25692E5A2A3B392E4201608A25992E1C2
:10358000A22692E0F608748020161220640FE551FE
:1035900054074480A25892E5A2A1B392E4F60874BD
:1035A00080F608F608F675F00778907E007F00E652
:1035B0002EFEE61234FAF62FFF08D5F0F2EED333E2
:1035C0001234FAF8EFD3336870647890B6FF5F0571
:1035D00061E56124FE501475610220180ED2187541
:1035E00018C0751900751A031209C4201608785EF0
:1035F000E2600330640302368E7896E620E35920B9
:10360000E24920E1277891E6B6002108B642090890
:10361000E6D263123ADE8076B6551108B6000D0880
:10362000794DE6F30809E6F3D252D2638060E56192
:103630006017D56114301811C2187518C0751900BB
:10364000751A041209C4757F0380437891863D087A
:10365000D25179A47A04800B7891D2507571057992
:10366000987A05D26375F00FE6C4540FF755F0F55C
:10367000F009E6540FF755F0F5F00908DAEAE5F03D
:10368000B40F051977EEC250785EE212342412347A
:10369000E022D293C2B4D2B21234BCC2931234CD5F
:1036A000D2931234CD20161F306323789076110800
:1036B0007480F608A2A3B392E4F6749008F608F6B4
:1036C00008F608F6023717789076150236D2789009
:1036D0007613087680087480A25692E5A2A3B3926E
:1036E000E4206314A25792E1A2A4B392E02016084A
:1036F000A25992E1A22692E0F608748020630FE5B9
:103700005154074480A25892E5A2A1B392E4F6086E
:103710007480F608F608F675F00778907E007F0052
:10372000E62EFEE61234FAF62FFF08D5F0F2EED3BD
:10373000331234FAF8EFD3336870627890B6FF5DD5
:103740000560E56024FE501475600220190ED21940
:103750007518C0751900751A051209C4785DE26004
:10376000033063030238087896E620E36520E255CB
:1037700020E1487891E6B6002208B6420A08E6D26F
:1037800064123ADE023808B6551108B6000D087901
:103790004DE6F30809E6F3D252D264806BE560602F
:1037A00017D56014301911C2197518C07519007534
:1037B0001A061209C4757F03023808D2647891860C
:1037C00040D24480437891863D08D25179A47A044E
:1037D000800B7891D25075710579987A05D264750D
:1037E000F00FE6C4540FF755F0F5F009E6540FF763
:1037F00055F0F5F00908DAEAE5F0B40F051977EEAF
:10380000C250785DE21234241234E022785EE26025
:103810001024FD400C75F0031282ECD5F0FA12353D
:103820003122785DE2601024FD400C75F0031282B5
:10383000ECD5F0FA12369222C0E030630C7518B065
:10384000751900751A001209C4D0E022D293C2B4CF
:10385000D2B21234BCC2931234CDD2931234CD788A
:1038600090E575540FC44407F608E57423A2E3926B
:10387000E5A2E292E3542AD2E7F608E574A2E392C5
:10388000E1A2E492E3542AD2E7F608E574A2E692B4
:10389000E1A2E792E3540AD2E7F6748008F608F64C
:1038A00008F675F00778907E007F00E62EFEE6129F
:1038B00034FAF62FFF08D5F0F2EED3331234FAF8CB
:1038C000EFD33368700B7890B6FF061234E0C380F4
:1038D000041234E0D3227575087873E2F574123857
:1038E0004C740040051239AC80031239D275750949
:1038F0007874E2F57412384C740140051239AC80CA
:10390000031239D22222E579542060F975750475C5
:1039100074FF12384C740250041239D2221239AC9E
:1039200078937948E6F30809E6F308794AE6F3085C
:1039300009E6F37891E6A2E092E25414F5F008E685
:1039400023A2E592E0540345F0F5F0784CE265F0EF
:10395000C0E0E5F0F2D0E030E21FC0E0C0F0E5F0FA
:1039600075F04930E20375F04A7518C07519008585
:10397000F01A1209C4D0F0D0E0540370030239AB3E
:10398000E5F05403B4030575F0488013B4020575DF
:10399000F047800BB4000575F04B800375F04C7553
:1039A00018C075190085F01A1209C422F5F02442D6
:1039B000F8E2B40205227402F22250FA7402F2E52F
:1039C000F02432F5F07518C075190085F01A120947
:1039D000C422F5F02442F8E2601AD5E016F2E5F0D0
:1039E000243CF5F07518C075190085F01A1209C449
:1039F000757F03F222D293C2B4D2B21234BCC29306
:103A00001234CDD2931234CD7890E575540FC4445E
:103A100003F6087680087480A25692E5A2A3B392BA
:103A2000E4A25992E1A22692E0F6087480A258928C
:103A3000E5A2A1B392E4F6087480F608F608F675DC
:103A4000F00778907E007F00E62EFEE61234FAF64C
:103A50002FFF08D5F0F2EED3331234FAF8EFD33358
:103A60006870717890B6FF6C7896E620E33020E2BB
:103A70002020E1607891E6B6005A08B6551108B6E4
:103A8000005208794DE6F30809E6F3D252804A80E5
:103A9000437891863D08D25179A47A04800B7891BD
:103AA000D25075710579987A0575F00FE6C4540FF8
:103AB000F755F0F5F009E6540FF755F0F5F0090861
:103AC000DAEAE5F0B40F051977EEC2507864E21235
:103AD000342480051234E0D3221234E0C322B4FF30
:103AE00015D270756F051238387518C075190075C4
:103AF0001A071209C422B4BC03023B0FB4BD03026F
:103B00003B41B4BE03023B73B4BF03023BA522207A
:103B100063147408F97480F87530017531CE75320C
:103B20004012043D80127408F97480F875300175F4
:103B300031CE75324812043D74117888F6123BD7A5
:103B4000222063147408F97480F87530017531CE41
:103B500075325012043D80127408F97480F8753083
:103B6000017531CE75325812043D74127888F61200
:103B70003BD7222063147408F97480F875300175FE
:103B800031CE75326012043D80127408F97480F8E9
:103B90007530017531CE75326812043D7413788822
:103BA000F6123BD7222063147408F97480F875303C
:103BB000017531CE75327012043D80127408F974AB
:103BC00080F87530017531CE75327812043D741469
:103BD0007888F6123BD7227881E6120158400474A7
:103BE0001ED3227882E61201A8400C741FD3221241
:103BF0006BEF1200D7C3227880E660F9B4FF08D2D9
:103C000070756F05023DF9B40212203A031238387C
:103C10007888E61221CB400280DB80D3B4090CC047
:103C2000E07404127E10D0E0023DF9B438087883C5
:103C3000E6123E0A80BFB439087883E6123E14804B
:103C4000B4B43A2530742012383878B2E278B3F23E
:103C5000788886F07518C0751909E5F0543F4480DE
:103C6000F51A1209C48088808CB43B223074F81293
:103C70003838E478B3F2788886F07518C075190979
:103C8000E5F0543F4440F51A1209C4023BEFB43C3E
:103C90000D1238387888861A122304023BEFB43D9F
:103CA0002B123838204311D24375187075190F75CF
:103CB0001AE91209C4023BEFC24375186075190F67
:103CC000751AE91209C4125287023BEFB43E13E59C
:103CD000795410600A123838E4123E19023BEF02A0
:103CE0003BF5B43F14E5795410600B12383874FF7B
:103CF000123E19023BEF023BF5B4400D1238387802
:103D000088861A122234023BEFB4410D12383878FB
:103D100088861A122275023BEFB4420D12383878A9
:103D200088861A12225C023BEFB4430D12383878B1
:103D300088861A12224D023BEFB4440E7400127EA4
:103D4000107888E6128338023BEFB4450E740012F7
:103D50007E3C7888E6128347023BEFB44609740044
:103D6000127E5940E880D5B4470E7402127E107856
:103D700088E6128356023BEFB4480E7402127E3C72
:103D80007888E6128365023BEFB449097402127E1B
:103D90005940E880D5B44A0E7403127E107888E644
:103DA000128374023BEFB44B0E7403127E3C78888E
:103DB000E6128383023BEFB44C097403127E594030
:103DC000E880D5B44D181283927888E6543F448039
:103DD000F51A75190B7518C01209C4023BEFB44EE1
:103DE0000C304306123838023CB8023BEFB44F099E
:103DF0002043F7123838023CA71238387518C075BE
:103E00001907F51A1209C4023BF51222937888E6C5
:103E100078AEF22212229D80F47873F208F2123802
:103E2000D67888E6543F44C0F51A75190B7518C04A
:103E30000209C4700575631E8002D21122C298C2A5
:103E400099322016F830991EC299204F0575350019
:103E50008014C0F0C0E0C0D075D010E53512416DBF
:103E6000D0D0D0E0D0F020980132C298204FFAC0D4
:103E7000F0C0E0C0D075D010304E05C24E75410084
:103E8000E54524FE4003754502E54120E71FE54175
:103E9000540723242FC0E074003440C0E0E5992289
:103EA00005412544F544D0D0D0E0D0F032543F2332
:103EB000232430C0E07400343FC0E0E5992215624D
:103EC00080DE80DCD562FBB54412D20FE8C0E0781A
:103ED000A974FAF2D0E0F875410080CA02403FB4FC
:103EE00062FA80BC80BAB42AF380B5F56224C6E5D4
:103EF0006240E924F5E56250E3056280A37818F298
:103F00001562809C7819F215628095781AF2156214
:103F1000808E781BF215628087781CF21562808093
:103F2000781DF21562023EA0781EF21562023EA0D4
:103F300002405700023EDF00023EE400023EE6007F
:103F4000023EEB00023EBE00023EBE00023EBE004C
:103F5000023EBE00023EFD00023F0400023F0B0095
:103F6000023F1200023F1900023F2000023F2800DA
:103F7000023EC400023EC400023EC400023EC40031
:103F8000023EC400023EC400023EC400023EC40021
:103F9000023EC400023EC400023EC400023EC40011
:103FA000023EC400023EC400023EC400023EC40001
:103FB000023EC400023EC400023EC400023EC400F1
:103FC000023EC400023EC400023EC400023EC400E1
:103FD000023EC400023EC400023EC400023EC400D1
:103FE000023EC400023EC400023EC400023EC400C1
:103FF000023EC400023EC400023EC400023EC400B1
:10400000023EC400023EC400023EC400023EC400A0
:10401000023EC400023EC400023EC400023EC40090
:10402000023EC400023EC400023EC400024057806B
:104030000E802D803180358038803B80488046B4AA
:104040000909754400754100023EA0B44209754457
:1040500000754180023EA0754400754100023EA6F5
:10406000B51EDC023EA0B51FD6023EA0F542023EC0
:10407000A0F543023EA0B544C675452012408775A1
:104080004100023EA680D0854237127327D24FE509
:1040900037B44603025968B4470412733D22B45042
:1040A0000E854336127302C2ACC24F75730722B439
:1040B0005312854336E543700A127302C2ACC24FF5
:1040C00075730222B4540E854336127302C2ACC219
:1040D0004F75730122B4550E854336127302C2AC7C
:1040E000C24F75730322B4560E854336127302C253
:1040F000ACC24F75730422B4570E85433612730257
:10410000C2ACC24F75730522B4580E854336127384
:1041100002C2ACC24F75730622B44E3D854336E5EC
:1041200043B4000B127302C2ACC24F75730822B4C1
:10413000010B127302C2ACC24F75730922B4020B99
:10414000127302C2ACC24F75730E22B4030B12730A
:1041500002C2ACC24F75730F2224BF24E64004850F
:10416000433622C24F22C5382538C53822E53524CA
:10417000F0400EE53523248CC0E074003441C0E0EB
:1041800022759906C24F753500D2B622802F803431
:10419000803680388039803E804680488051804F0C
:1041A000804D804B80468050800E0242347535032E
:1041B000F599124166053522E5360241E27538006F
:1041C000740380ECE51E80E8E51F80E4024298E578
:1041D0003875350F80DA120A02123E33883680D0E5
:1041E000E53680C9E536A24392E080C1753503A863
:1041F000360536E676FF80B8E536C31360321470B4
:104200000BA22392E0B392E1440480D614700BA277
:104210002492E0B392E1440880C8147008A2259269
:10422000E0440C80BD147008A22B92E0440C80B2D4
:1042300074FC80AEE5361470257408305C12305D75
:10424000044406809D305E044403809644078092B7
:10425000A25D92E0A25E92E1A22692E280841470B6
:10426000157410A22392E0A22492E1A22592E2A268
:104270002B92E30241E214700D7418A21892E0A28E
:104280001992E10241E214700BA25F92E0A26192E6
:10429000E20241E2E40241E2E537B4410675350449
:1042A0000241B0B44212E5366003301103120A1A1B
:1042B00075631E74420241ADB4440280F8B44B02EF
:1042C000800302435DE53654F8B4083EE5365407F2
:1042D000700B751A19122234E537024392B4010BA0
:1042E000751A1912224DE537024392B4020B751A62
:1042F0001912225CE537024392B4030B751A1912A6
:104300002275E537024392024181B42003024181C4
:10431000B42826E53620E00830430B125287800689
:10432000204303127553E536A2E09243756E0150A7
:1043300003756E02E5370241ADB4300CE53654F832
:10434000127E10E5370241ADB4380CE53654F81250
:104350007E3CE5370241AD024181024181B4430F09
:10436000B536037546037535077536AC0241B0B4F2
:104370004A26E536701F205E1C205C087419126EF8
:1043800097126E8575181075190F751AF01209C4F9
:10439000E5370241AD024181B4450675350602415B
:1043A000B0B4510675350C0241B0B44D0EE536126D
:1043B0008120E5375002B2E70242B5B44C067535AC
:1043C0000E0241B0B4460280C9B4470280C4B44F63
:1043D00008C245C246C24780B9B4590FE536700BD2
:1043E000857E36745975350D0241B0024181E57301
:1043F000B4000122B40717C2AC12831C12831CD272
:1044000099127169C24FD2B6127302024512B401F9
:1044100017C2AC12831C12831CD299120FC5C24F53
:10442000D2B6127302024512B40317C2AC12831C37
:1044300012831CD29912104AC24FD2B612730202D2
:104440004512B40217C2AC12831C12831CD29912FB
:104450000EE6C24FD2B6127302024512B40417C25E
:10446000AC12831C12831CD299120F28C24FD2B6F1
:10447000127302024512B40517C2AC12831C1283D8
:104480001CD2991202ACC24FD2B61273020245126C
:10449000B40617C2AC12831C12831CD2991210925C
:1044A000C24FD2B6127302024512B40817C2AC1240
:1044B000831C12831CD299126D2FC24FD2B6127375
:1044C00002024512B40917C2AC12831C12831CD21B
:1044D00099126CB3C24FD2B6127302024512B40ED7
:1044E00017C2AC12831C12831CD299126DBCC24F2E
:1044F000D2B6127302024512B40F17C2AC12831C5B
:1045000012831CD299126DFEC24FD2B612730202F0
:10451000451275730022E565C2676002D267E552F5
:10452000F553C24820520C20501B30510302464B19
:10453000024B16120102784DE2F58308E2F5821271
:104540001A48024708120102121CA8121B326017F7
:10455000121BC2603C12383875182075190F751A75
:10456000EC1209C4024594206305205F0A800320F1
:104570006105124BC2501AC082C0831200E412209F
:10458000CBD083D08230510CE53D60081219D27037
:1045900003024708754A3CD546177518C0751900BF
:1045A000751A531209C4754603757D00D2467549C4
:1045B000B4024B03D270756F051238387518C07588
:1045C0001900751A071209C475510412380C1238F3
:1045D0002275F06412011E024B16206324E57B5401
:1045E0000860CE300818C0E0C082C0837411120188
:1045F00088D083D082D0E0400280B90246220246B1
:1046000022E57A548060AA300818C0E0C082C083D6
:104610007410120188D083D082D0E04002809502CD
:104620004622122348401E205E15302E03204309E7
:10463000900FE9124B1F024B16124AA0024B1612A2
:104640004AA6024B16124AAC024B16120102E53D75
:10465000608878A4E6B40A03025279121C0B707DBC
:10466000206305205F50800320614B124BC24046FF
:10467000206325300819C0E0C082C0837413120182
:1046800088D083D082D0E0400302470802469202DD
:104690004708124A7C024594300818C0E0C082C026
:1046A000837412120188D083D082D0E04003024785
:1046B0000880DF0247081200E4C082C0831221593B
:1046C000D083D082305013C082C083120102121CEA
:1046D000A8D083D082121910602E024594785D20F4
:1046E0006402785EE2B40F0A124EADC251D250029B
:1046F0004548B4100280F112383875182075190F2A
:10470000751AEB1209C480D2306330300819C0E04A
:10471000C082C083740C120188D083D082D0E04064
:104720000302473B024727757502785FE27864F21F
:104730001214901250265003024594306430300811
:1047400019C0E0C082C083740D120188D083D0826A
:10475000D0E0400302476E02475A7575037860E265
:104760007864F212149C125026500302459412747D
:10477000FD40031234B3E53C047003024594754ACE
:1047800000754603C247C246204802C245C082C0E7
:1047900083124C69D083D0825006124ABB024B165A
:1047A000C082C0831205DBD083D0825006124ABB80
:1047B000024B16E58224CEE58334FF5017124BB02E
:1047C0004012C212C2131232AF5006124AAC024B50
:1047D000160249B71223485012124AAC02495B1222
:1047E0004AA602495B124AA002495B205EF1302EC4
:1047F000032043F13063037854E2306402E53C1255
:1048000001584003024810024854124A9A02495B78
:104810003008F73014F4303DF112517D4036A26378
:10482000303E01B3502E300818C0E0C082C08374FF
:1048300009120188D083D082D0E0400280CC0248A7
:1048400041C082C0831270F5D083D0825006124AD4
:10485000B102495B301425D239300819C0E0C0825A
:10486000C0837414120188D083D082D0E040030248
:104870004877024875C23912517D50030248EC1244
:1048800070A1A2E09212A2E19213A263303E01B3A2
:10489000C0E09206501E12714B501930390EE4A23E
:1048A0001292E0A21392E1B402028008D0E0124A10
:1048B0008802495BD0E0B40005200622802BB401B9
:1048C0002220061A7518C0751900751A091209C434
:1048D000203906124AB602495B124B73800E126FE2
:1048E000F48009B402ED2006DB12704C3008581237
:1048F000517D4053300819C0E0C082C08374081253
:104900000188D083D082D0E0400302494702491099
:1049100020671AA2639266858366858267124B6F51
:10492000C263C2641200F8756502024B1675650019
:10493000E5836566F5F0E582656745F07006124A25
:10494000C002495B12521A124B1FE5795410600BDA
:10495000C082C083124D79D083D082124BB95009E6
:10496000124D5330E103024B161232AF40F8C2A190
:10497000D258D2A4C25775510012380C12382212E4
:104980001A48C082C083122159D083D08220520994
:1049900020501720511C024B16120102784DE2B52F
:1049A000830D08E2B582080249B7121910600802A7
:1049B0004B031219D270F8301424E4A21292E0A230
:1049C0001392E1B403051270788013B40205126FDC
:1049D000F4800BB4010512704C8003126FCB3008C9
:1049E00019C0E0C082C0837406120188D083D082CF
:1049F000D0E04003024B030249FAE57954016022FA
:104A0000E5824583601C3063037854E2306402E53C
:104A10003C1201584003024A1C024A22124A8E02EA
:104A20004B1612235B500F124A9475F01E12011E92
:104A30001200C1024B16B24312383830431D7518AC
:104A40007085831985821A1209C4C2A3C256D2A1E5
:104A5000C258D2A4C257127553801B751860858343
:104A60001985821A1209C4D2A3C256D2A1C258C251
:104A7000A4C2571252871200D7024B16126BE502DE
:104A80004AC3126BE5024AC3126BE5024AC3126BBA
:104A9000E5024AC3126BE5024AC3126BE5024AC340
:104AA000126BE5024AC3126BE5024AC3126BE58042
:104AB00012126BE5800D126BE58008126BE5800326
:104AC000126BE57565007566FF7567FFD277123862
:104AD0003875182085831985821A1209C41200C1FD
:104AE000C27722E57A54087003206316E552046009
:104AF00011146564600C7518C075190185521A127D
:104B000009C422126BE5D2771200ABC2777565003B
:104B10007566FF7567FFC251C250E553F5522230EA
:104B2000430EC2A3C256C2A2C259D2A4C257800C1D
:104B3000D2A3C256C2A2C259C2A4C257A263920A49
:104B4000D209126BE5741C126E97126E85E57954CA
:104B500040600620A80312337C123838124AE375ED
:104B6000181085831985821A1209C41200D72212DF
:104B70006BE522126BE575F03212011E227408F902
:104B80007480F875300175310375329012043D78E8
:104B900085E6085608560460141200E41220CB3053
:104BA0005109E53D60051219D26002C322D32222C9
:104BB000E582249CE58334FF22E582249CE583344E
:104BC000FF22A240E58245836010E582249CE583B4
:104BD00034FF5004A23F8002A24122E5822582F5E3
:104BE00082E5833583F583E5822582F582E5833589
:104BF00083F583E5822400F582E583345BF58374D5
:104C000004F97400F875300185833185823212040D
:104C100018227885E654C0F5837886E630E40224CD
:104C20000A2323543C4583F5837885E6C4540375F1
:104C3000F00AA4F5F0E6540F25F0030303F5F05352
:104C4000F0E085F08254034583F5837884E6C4540C
:104C50000375F00AA4F5F0E6540F25F04582F582BD
:104C600022C39582E5F095832212517D5003024CB8
:104C7000F1124BDB7800E2B4FF03024CF11277CF64
:104C8000124C127880A68308A6827800E2F5830889
:104C9000E2F58208E2F5F008E2124C61502B780050
:104CA000E2F58308E2F582788086F008E6124C612E
:104CB00050417802E2F58308E2F582788086F008B8
:104CC000E6124C61402D024CF17800E2F58308E2D7
:104CD000F582788086F008E6124C6140167802E290
:104CE000F58308E2F582788086F008E6124C615080
:104CF00002C322D322C3E58233F582E58333F583F1
:104D0000E5822400F582E583349AF5837402F97410
:104D100053F875300185833185823212041822C31D
:104D2000E58233F582E58333F583E5822400F5825D
:104D3000E583349AF5837402F97453F8753001856C
:104D400083318582321203612278537400F208E4C1
:104D5000F2801E3008F3C082C083124CF5D083D09D
:104D600082E5822418E58334FC40067853E244024D
:104D7000F27854E2F5F018E222E5822400F582E5AB
:104D80008334BAF5837401F97480F8753001858332
:104D90003185823212043D7880E660422323C0E0F0
:104DA0005403F5F0D0E054FC2400F582E5F034CA59
:104DB000F5837404F97480F8753001858331858238
:104DC0003212043D7880E60886F07873F208E5F048
:104DD000F275F0021282ECD5F0FA1238D62274FF86
:104DE0007873F208F280EAE572B4220575F0048067
:104DF00013B42A0575F006800BB4420575F00C80DB
:104E00000375F002782EE2540F704F08D5F0F7E2E8
:104E1000540F75F00AA4F58275830008E2540F253B
:104E200082F582E58275F00AA4F58285F08308E2B6
:104E30002582F58250020583E58275F00AA4F58289
:104E4000C0F0E58375F00AA4D0F025F0F58308E200
:104E50002582F58250020583C322D322782EE26098
:104E60000BF5F008E2240A4005D5F0F7C322D3225F
:104E7000782EE572B4220A757104799A75F008806B
:104E800024B42A0A757105799875F00A8017B4421E
:104E90000C757105799875F00A783480087571037E
:104EA000799C75F006E2F70809D5F0F922C082C0B6
:104EB0008378989002E075F00AE0F608A3D5F0F93F
:104EC0009002EAE0F571D083D08222C082C083785C
:104ED000989002E075F00AE6F008A3D5F0F9E571C4
:104EE0009002EAF0D083D08222124E701219102262
:104EF000D083D08222124E70124ECB122139C08242
:104F0000C083753D01782EE2540F70E408E2540F1F
:104F100070DE08E2540FC4F5F008E2540F45F0F5D6
:104F20008308E2540FC4F5F008E2540F45F0F5820F
:104F3000C26D78A47900C3E5829410F582E583946C
:104F400027F58340030980EEE5822410F582E5838E
:104F50003427F583E96004D26DF6087900C3E58251
:104F600094E8F582E5839403F58340030980EEE538
:104F70008224E8F582E5833403F583E9206D04603B
:104F800004D26DF6087900C3E5829464F582E58366
:104F90009400F58340030980EEE5822464F582E500
:104FA000833400F583E9206D046004D26DF608E5D2
:104FB0008275F00A84206D026002F608E5F0F6E8DA
:104FC000245DF53DD083D0822279A477000975F065
:104FD0000577FF09D5F0FA22124E70124ECB124F10
:104FE000C975F008E572B42204782E8013B42A043F
:104FF0007830800CB4420478368005782E75F0063F
:10500000753D06E2540F700608D5F0F7800979A4C3
:10501000E2F70809D5F0F922124FD81219D222125C
:105020004EF51219D2227864E270030250DB24FD9F
:105030004038C082C0831200E4125137D083D0823E
:1050400020521620510B3050361219107031025078
:10505000DB1219D270290250DB784DE2B5832008AB
:10506000E2B5821B658270178071E224E24070C055
:1050700082C0831200E4127994D083D0825003025C
:1050800050DD7864E2B40F0C125018604E124EE9F5
:10509000604980EBB4100712501F603F80E175F04B
:1050A0000384E5F0B4000712501870D3802DB401CA
:1050B00007124EE970C98023B4021EC082C0831259
:1050C0004DE7E5828583F0D083D08240B26582705F
:1050D000AEE5F0658370A8800280A4C322D322C00D
:1050E00082C0831200E41279EAD083D0825002D3C6
:1050F000227864E275F00384E5F0B4000A12518B63
:105100001219D270EA802CB4010A1251B31219108C
:1051100070DD801FB4021EC082C0831251B6E582CA
:105120008583F0D083D08240C6658270C2E5F06589
:105130008370BCC32280B8754832D25B305409C238
:1051400054C07512027AD075E548D36018C252C2B5
:1051500051C250121F9650E41239F52052062051C8
:10516000033050D8C3C0D0A8757405B802027404C7
:10517000D0D040051239AC80031239D222E582B476
:10518000E807E583B40F02D322C322124E5C50021B
:10519000D322782EE260F9F5F008753D06E2540F4F
:1051A000700608D5F0F7800979A4E2F70809D5F070
:1051B000F9C322027B0C124E5C5004D322C3227826
:1051C0002EE20860F6B40108E2F58275830080EDF6
:1051D000B40212E275F00AA4F58208E22582F58293
:1051E00075830080D8B40320E275F00AA4F5820824
:1051F000E2258275F00AA4F58285F08308E2258213
:10520000F58250B9058380B5B40405782F024E0F9E
:10521000C39404F5F0782F024E06B263B264755160
:105220000712380C123822B264B2637518C07519AF
:1052300000751A0C1209C430660C7518B075190087
:10524000751A001209C4124AE3751810856619858B
:10525000671A1209C422E53DB4031C78A4E6B40A17
:105260001608E624F6401008E624F6400A18E6750B
:10527000F00AA40826C322D3221252565003024633
:105280005B78ACF20252D6127553128392C245C2B9
:105290004822532D534F538B53B753CE53E553FCF2
:1052A0005413542254315440544F548354AB54B388
:1052B00054C554D45510555F5582559955BA55D695
:1052C00055F255FE561A56365642565E567A568650
:1052D000569F5301530178ACE224E040241257E872
:1052E000401378ACE225E00490529293C0E0E225AE
:1052F000E093C0E0220258A012589F1200D7024B40
:1053000016740A0258A0D2A1C258C2A4D257125889
:105310009E1200E4122159205102D322E53DB4022D
:10532000F978A4E624F640F208E624F62212589D05
:10533000125306401578A4E62430F51E08E6243002
:10534000F51F1218EA12665F80AE74200258A01290
:10535000589D125787402F1277CF78A4E6C408468D
:10536000F5F078A8E65403030345F07885F678A6AF
:10537000E6C40846F5F078A9E6C42345F07886F639
:105380001277B00252F8741E0258A012589D12579C
:1053900038401F1277CF78A4E6C408467884F678A0
:1053A000A6E6C408467883F6E47882F61277B0025F
:1053B00052F8741F0258A012589D1258817518C0D7
:1053C000751900751A0F1209C4D25F0252F81258EB
:1053D0009D1258817518C0751900751A101209C4EC
:1053E000C25F0252F812589D1258817518C0751983
:1053F00000751A511209C4D2610252F812589D1256
:1054000058817518C0751900751A521209C4C26105
:105410000252F812589D125881751A1B122234023A
:1054200052F812589D125881751A1B12224D0252C1
:10543000F812589D125881751A1B1222750252F8E3
:1054400012589D125881751A1B12225C0252F812D2
:10545000589D1232AF402712588112755312839211
:10546000C245C248C243784DE2F58308E2F5827531
:10547000186085831985821A1209C40252F87416BD
:105480000258A012589D1232AF40F3125881127583
:1054900053D243784DE2F58308E2F58275187085A2
:1054A000831985821A1209C40252F812589D2043AA
:1054B0009E80D012589D12588175F0C81282ECD58A
:1054C000F0FA0274D012589D125881751A1B1223DB
:1054D000040252F812589D20150D125700402C124C
:1054E00058B3402778ADF278ADE2F552F553125833
:1054F000817518C085521A75190330150375190284
:105500001209C40252F874190258A0741A0258A061
:1055100012589D20150D12570040F01258B340EB61
:1055200078ADF278ADE2F5521258817518C0855207
:105530001A7519063015037519051209C41268FC8D
:10554000124BAFD2A2C259C2A1D2581200E412210A
:105550005974182050062051033052B102452412CC
:10556000589D30742D78B2E278B3F21258817518D4
:10557000C0751909741B543F4480F51A1209C402FE
:1055800052F812589D30740A125700500A741C02C7
:1055900058A0741D0258A070CF12589D3074F3E4C7
:1055A00078B3F21258817518C0751909741B543FED
:1055B0004440F51A1209C40252F812589D740012A0
:1055C0007E107518C075190A741B543F4400F51AF3
:1055D0001209C40252F812589D7400127E3C7518CC
:1055E000C075190A741B543F4480F51A1209C4028D
:1055F00052F812589D7400127E5940DD80BF125837
:105600009D7402127E107518C075190C741B543FDE
:105610004400F51A1209C40252F812589D7402127D
:105620007E3C7518C075190C741B543F4440F51A24
:105630001209C40252F812589D7402127E5940DDBC
:1056400080BF12589D7403127E107518C075190C16
:10565000741B543F4480F51A1209C40252F81258C0
:105660009D7403127E3C7518C075190C741B543F51
:1056700044C0F51A1209C40252F812589D7403125C
:105680007E5940DD80BF7404127E107518C07519F4
:105690000B741B543F4440F51A1209C40252F8120D
:1056A00083927518C075190B741B543F4480F51A0A
:1056B0001209C40252F8C2A1D258C2A4D257124B46
:1056C000AF1200E412215920520820501C20512909
:1056D000D322784DE2F58308E2F582120102300808
:1056E00006124D5320E2E9C322121B3270E2784DBC
:1056F000E583F208E582F280E2121C0B70D280EEA4
:10570000D2A1C258C2A4D25712589E1200E412214C
:1057100059205102D322E53D60FA24FC40F6A93D10
:1057200078A47A00EA75F00AA42640E8C5F070E48F
:10573000AAF008D9EFEAC322D2A1C258C2A4D25714
:1057400012589E1200E4122159205102D322E53D45
:10575000B404F9F5F078A4E624F640F008D5F0F7A3
:1057600078A4E675F00AA4082624E8402E78A6E678
:1057700075F00AA4082624C4402122E0E2E0E1E01A
:10578000E1E0E0E1E0E1E0D2A1C258C2A4D25712C8
:10579000589E1200E4122159205102D322E53DB453
:1057A00006F9F5F078A4E624F640F008D5F0F7788D
:1057B000A6E675F00AA4082660E1C0E024F3D0E074
:1057C00040D990577A93F978A4E675F00AA4082690
:1057D00060C9C0E029D0E040C278A8E624F640BB0A
:1057E00078A9E624F940B42230087C784D740FF291
:1057F0000874E9F220157C78ACE22400F582758308
:10580000D07401F97480F875300185833185823256
:1058100012043D7880E6120158506278ACE2240010
:10582000F5827583D17401F97480F8753001858330
:105830003185823212043D7880E61201A850367814
:10584000ACE22400F5827583CF7401F97480F87599
:10585000300185833185823212043D7880E62063F1
:105860000C20E01530E10C1256B6740D2220E2092E
:1058700020E3F4C322740E8006740C8002740BD3F0
:1058800022201518123838784DE2F58308E2F582A7
:105890007518E085831985821A1209C422222222F2
:1058A000C0E0126BE512589DD0E01267DC1200AB2D
:1058B000024B16C052C082C083F55212685FD0837B
:1058C000D082E552D052B322C5382538C53822E5FA
:1058D0004A24E94008D2A3C256D2A2C2593098EF56
:1058E000C298E5991258C8223099FDC299F59912CB
:1058F00058C822C2A3C256C2A2C259C2B675380045
:1059000074051258E8E51E1258E8E51F1258E822FF
:1059100012831C12831C12831C1258F3E537125891
:10592000E8E5381258E83099FD221209320259335D
:105930001208CEC0E01258F3E5371258E8D0E01252
:1059400058E8E5381258E83099FD2212831C1258A5
:10595000F3E5371258E87980E71258E809DDF9E5F0
:10596000381258E83099FD22D216754A19751A0076
:10597000128392E539600B54F87007C227A227B34F
:1059800092A5E53A600B54F87007C228A228B3929A
:10599000A6E53B600B54F87007C22CA22CB3928092
:1059A000126E92C28EC28CC2ADC2ABC2ACC2AF7517
:1059B00081D79059BDC082C08375D00032D2AFD29A
:1059C0008C127302C2ACD299125910B2B5754A1931
:1059D000D2980259FAB40922F5381258CFB51E27C9
:1059E0001258CFB51F211258CFB4461B1258CFAF53
:1059F000381258CF6F7010125910D2B6D2A3C256B7
:105A0000D2A2C2591258CFB40ACBF5381258CFB52A
:105A10001EF51258CFB51FEF1258CFF537B46D03EE
:105A2000025AB0B46E03025AC9B46F03025B00B4E9
:105A30007003025B4DB47103025B61B47303025BDC
:105A400072B47403025B74B47503025B88B47603AA
:105A5000025BA0B47703025BA3B47803025BB7B424
:105A60007903025BD8B47A03025BF4B46C03025C82
:105A700008B46B03025C2AB46A03025C65B4690370
:105A8000025C81B46803025CE0B46703025CF8B4B2
:105A90006603025D13B46503025DD7B46403026557
:105AA0001BB463030264E2B461030265760259FA2F
:105AB000AF381258CF6F70F5125910D2B675F01E6C
:105AC0001282ECD5F0FA0274D01258CFFD1424E003
:105AD000402B1258CF2400FC7B001258CFFEAF3869
:105AE0001258CF6F70178EF0EDF97480F88B308CF0
:105AF0003185F03212043D12594B754A190259FA98
:105B00001258CFFD1454E070F41258CF2400FC2436
:105B10007140EA7B021258CFFEEDFA78801258CF1E
:105B2000F608DAF9AF381258CF6F70D1C2A3C25657
:105B3000C2A2C2598EF0EDF97480F88B308C318599
:105B4000F032120392125919754A1980B0AF381207
:105B500058CF6F70A81206F2125910754A190259DF
:105B6000FAAF381258CF6F7009125930754A1902BE
:105B700059FA80891258CFFD1424E040371258CFCB
:105B80002400FC7B01025ADA1258CFFD1454E07055
:105B9000231258CF2400FC242540197B03025B15F7
:105BA000025AFDAF381258CF6F700912592A754A40
:105BB000190259FA025AFD79187D071258CFF309D4
:105BC000DDFCAF381258CF6F70EA1267DE40E51285
:105BD00077B01259190259FAAF381258CF6F70D4F2
:105BE0001277CF12831C1258F3E5371258E81202CD
:105BF000C80259FAAF381258CF6F7066120CD01223
:105C00005910754A190259FA1258CFFE1258CFFD91
:105C10001258CFFCAF381258CF6F7046120658405A
:105C200041125910754A190259FA1258CFFE1258EA
:105C3000CFFDAF381258CF6F702812062912831C7F
:105C400012831C1258F3E5371258E8EE1258E8EDAB
:105C50001258E8EC1258E8E5381258E83099FD027D
:105C600059FA025AFDAF381258CF6F70F512831CE3
:105C700012831C1258F3E5371258E81210AB025980
:105C8000FAAF381258CF6F70D91208C6600274018B
:105C9000C0E012092A60027402D0F045F0700A12C6
:105CA000073D121548120CD0E4C0E01258F3E53756
:105CB0001258E8D0E0C0E01258E8E5381258E8750C
:105CC000F0031282ECD5F0FA1258F3E5371258E8D7
:105CD000D0E01258E8E5381258E83099FD0259FA38
:105CE0001258CFFD1454E070271258CF2400FC2422
:105CF00071401D7B00025B151258CFFD1454E070FB
:105D00000F1258CF2400FC242540057B01025B15AF
:105D1000025AFDAF381258CF6F70F512831C1283F0
:105D20001C1258F3E5371258E874021258E8744E02
:105D30001258E874801258E874481258E874321205
:105D400058E874001258E8748D1258E874201258FC
:105D5000E874DA1258E874001258E8740F1258E820
:105D600074A01258E874801258E874001258E8744D
:105D7000001258E874201258E874001258E87400B1
:105D80001258E874001258E874001258E8740012AF
:105D900058E874001258E874001258E87400125859
:105DA000E874001258E874001258E874001258E8B9
:105DB00074001258E874001258E874001258E8741D
:105DC000001258E874001258E8E5381258E8309983
:105DD000FD0259FA025AFD1258CFF5831258CFF539
:105DE000822460E58334F040EB1260631258CFFDEB
:105DF0001454E070DF780075F02074FFF208D5F0DD
:105E0000FB78001258CFF208DDF9AF381258CF6F87
:105E100070C212591075F0051282ECD5F0FA1259C1
:105E200019751A013008AD12609912607F12607105
:105E3000121A48789879007A0A75F00FE3540FF631
:105E400052F00809DAF643F0F0E5F00478A179841D
:105E50007A05121923600B125EF85006751A0402B7
:105E60005DD412607F126071121A4878A4790A7AA0
:105E70000675F00FE3540FF652F00809DAF643F016
:105E8000F0E5F00478A979877A03121923600B12E0
:105E90005F965006751A06025DD412607F1260E2AA
:105EA000751A650259FAC0E07828E583F208E582A0
:105EB000F2D0E022C0E0782AE583F208E582F2D051
:105EC000E022C0E07828E2F58308E2F582D0E02203
:105ED000C0E0782AE2F58308E2F582D0E022E5828C
:105EE0002400F582E583341BF58322E5822400F546
:105EF00082E583343BF58322126071AB83AC8290E0
:105F00001B00C083790075300385833175320090A2
:105F100000551203471204B81203471205169000E9
:105F2000557A80E0A3F5F0E0A36C7005E5F06B60B6
:105F300017DAF0D0830583740024C0E58334C5509C
:105F4000C17405126045D322D083EA2AF5F0E4C378
:105F500095F0F582125EA6789879007A0A75F00FAE
:105F6000E3540FF652F00809DAF643F0F0E5F004D6
:105F7000600C121B35700A7406126045D322121B86
:105F800035E5822582F582E5833583F583125EDE71
:105F9000125EB40262EA126071AB83AC82903B0085
:105FA000C0837900753003858331753200900055C8
:105FB0001203471204B81203471205169000557ACF
:105FC00080E0A3F5F0E0A36C7005E5F06B6017DAF4
:105FD000F0D0830583740024C0E58334A550C174D8
:105FE00005126045D322D083EA2AF5F0E4C395F088
:105FF000F582125EA678A4790A7A0675F00FE3544A
:106000000FF652F00809DAF643F0F0E5F004601DEF
:10601000121C1B701BAB83AC82126071EBB5830644
:10602000ECB58202C3227404126045D322121C1BF9
:10603000E5822582F582E5833583F583125EEB12D6
:106040005EB40262EAF51A22C082C083E583126759
:10605000DDD083D082C082C083E5821267DDD08329
:10606000D08222C0E0782CE583F208E582F2D0E00D
:1060700022C0E0782CE2F58308E2F582D0E02274B9
:10608000001258E874001258E874001258E87400BE
:106090001258E874001258E82275831B75821B752C
:1060A000F040C0F0C082C083753001858331753205
:1060B000001203471204B8D083D082C082C0837517
:1060C000300385823175320012034712057ED0837A
:1060D000D08205830582D0F0D5F0C77533FF7534C3
:1060E000FF227401F97418F87530007531007532AB
:1060F0000012043D7401F97419F87530017531D935
:106100007532FF12043DAC18126071E5822420F54F
:1061100082E583347DF583C082C0837401F9743CC9
:10612000F875300085833185823212043DD083D0EA
:10613000827401F97410F8753000858331858232DC
:106140001203617810E2F5F0E518253CC395F0F5EF
:1061500018126071124CF578537980E2F72519F521
:10616000190809E2F72519F51978167953E2F3FAB7
:106170000809E2F32AFAC3E5199AF51912607112B7
:106180004D1F126071E58275F008A42420F582503D
:106190000205F0A8F0E58375F008A4282400F58333
:1061A0007408F97480F87530008583318582321265
:1061B000043D7880E5187A082608DAFCF518789806
:1061C00079007A0A75F00FE3540FF652F00809DAF5
:1061D000F643F0F0E5F00412672178A4790A7A0614
:1061E00075F00FE3540FF652F00809DAF643F0F0B9
:1061F000E5F0041267297408F97480F87530008599
:1062000083318582321203927880E5187A08C3962A
:1062100008DAFBF518126071C3E58233F582E58375
:1062200033F583C3E58233F582E58333F583E58275
:106230002400F582E583245BF583C082C083740467
:10624000F97480F875300185833185823212043DFE
:10625000D083D0827404F97412F8753001858331CB
:1062600085823212036178807912E5197A0426F565
:10627000F0E3C5F0C395F00809DAF3F5197401F9F4
:106280007418F8753000753100753200120392747D
:1062900001F97419F87530017531D97532FF12039F
:1062A0009275831B75821B75F040C0F0C082C0835D
:1062B0007530038583317532001203471204B8D05C
:1062C00083D082C082C083753001858231753200EF
:1062D00012034712057ED083D08205830582D0F059
:1062E000D5F0C77533FF7534FF22125ED0E5828585
:1062F00083F0125EC2C39582C0E0E5F09583D0F0D2
:1063000045F07002C3225003026405125ED0C0E063
:10631000C3E58224FEF582E58334FFF583D0E012E5
:106320005EB4E5828583F0125EC2B58207E5F0B502
:106330008302C322125EC2AF83125ED0EFB5831018
:10634000AE8290002C7880E0F6A308E0F602636845
:106350007EFE8F8305837402F97480F8753003859F
:10636000833175320012043D79007530038F317529
:1063700032009000551203471204B8120347120569
:10638000168F83758200125EC27D00E5836F7002F6
:10639000AD82ED2455F58275830050020583C3EE6E
:1063A0009D20E05A03FCC082C083A3A3E0FAA3E0CF
:1063B000FBD083D082EAF0A3EBF0A3DCE9EE245516
:1063C000F582758300500205837880E6F0A308E625
:1063D000F079007530038F3175320090005512034B
:1063E0004712056A12034712057E85303385313422
:1063F000125ED0EFB583030264D90F0263397408CB
:10640000126045D322125EC2AF83125ED0EFB58315
:1064100010AE8290002C7880E0F6A308E0F60264CB
:10642000397E008F8315837402F97480F875300308
:106430008583317532FE12043D79007530038F314A
:106440007532009000551203471204B81203471228
:106450000516125EC27DFEE5836F7002AD82ED24EB
:1064600055F58275830050020583C3ED9E20E06BD5
:1064700003FCC0E0C3E58224FEF582E58334FFF52A
:1064800083D0E0C082C083E0FAA3E0FBA3EAF0A3DC
:10649000EBF0D083D082DCDAEE2455F582758300F0
:1064A000500205837880E6F0A308E6F079007530A5
:1064B000038F3175320090005512034712056A129E
:1064C000034712057E853033853134125ED0EFB537
:1064D00083030264D91F02640AC32274091260454F
:1064E000D3221258CFF5831258CFF5821258CF70AD
:1064F000271258CF7022AF381258CF6F701AC01EB3
:10650000C01F85831E85821F1218EA12665FD01F86
:10651000D01E1259100259FA025AFD1258CFF583B3
:106520001258CFF582AF381258CF6F70EBC01EC033
:106530001F85831E85821F1218EA7401F97480F882
:1065400075300075310075320012043D7880E6C365
:10655000951EC3951FD01FD01E251E251FF6740142
:10656000F97480F8753000753100753200120392AD
:106570001259100259FA1258CFF583AF381258CF7A
:106580006F709512831C12831C12831C1258F3E542
:10659000371258E874001258E8E51A1258E87400E7
:1065A0001258E874001258E874001258E874001287
:1065B00058E8E5381258E83099FD0259FA9065C557
:1065C000C082C083327581D775D0000274D0C0827A
:1065D000C083E5822420F582E583347DF583740150
:1065E000F9743CF87530008583318582321203924C
:1065F000D083D082C082C083E58275F008A42420B5
:10660000F582500205F0A8F0E58375F008A428246F
:1066100000F5837404F97480F87530008583318542
:106620008232120392A3A3A3A37404F97484F875AD
:106630003000858331858232120392D083D082E587
:10664000824583600EE5822418E58334FC74FFF5EF
:10665000F0500BC082C083124D1FD083D082221213
:1066600008CEC0E07401F97480F87530007531000F
:1066700075320012043D7880E6D0F0C395F0F674D0
:1066800001F97480F875300075310075320012031D
:106690009222753C007854E4F2788075F00876FF19
:1066A00008D5F0FA22751E30751F30C263C26475BA
:1066B000F005C0F0D2A3C256C2A2D259D2A1C2588C
:1066C000D2A4C257126692122159D0F0205009204C
:1066D0005106D5F0DD02671C126741403F1200D71A
:1066E0007885E6B4FF05C32275F005C0F012215984
:1066F000D0F0205106D5F0F302671CE53DB4021C32
:1067000078A4E624F6401508E624F6400F78A4E6BF
:106710002430F51E08E62430F51FC3221200ABD347
:1067200022789879807A05800678A479857A03E6BC
:1067300008540FC4F5F0E608540F45F0F709DAEFF6
:106740002220503130513AE53D600624FD24FC40C2
:10675000301267291200E475F005C0F0122155D0FF
:10676000F0205011204406D5F0F002678112115C30
:10677000B40B0E8003126721753C007854E4F2C319
:1067800022D32212679375F0641282ECD5F0FA12CC
:10679000007C2275F03C12011E126E8D75F03C12C9
:1067A000011E126E9275F01412011E126E8D75F09C
:1067B0003C12011E126E9275F01412011E126E8DA3
:1067C00075F01412011E126E9275F01412011E1251
:1067D0006E8D75F01412011E126E92222222781D07
:1067E000E254C07078E275F00A84C445F07882F60D
:1067F000781CE254C07066E275F00A84C445F078F3
:1068000083F6781BE254E07054E275F00A84C445C4
:10681000F07884F6781AE2604454E07040E275F053
:106820000A84C445F0C0E07818E2030354C0D0F0F5
:1068300045F07885F67819E2602354F0701FE27510
:10684000F00A84C445F0C0E0781EE254F8700EE20D
:10685000C42354E0D0F045F07886F6C322D32290CA
:10686000000075F019C0F07402F97480F8753001F9
:1068700085833185823212043D7881B6FF02800E15
:1068800018E552300805B4FF02E564666011E58240
:106890002410F58250020583D0F0D5F0C8C322D071
:1068A000F0A3D32230084DE58224FFF582E583343E
:1068B000FFF58375F019E5822480E58334FE5005E9
:1068C000900000800AE5822410F58250020583C002
:1068D000F07402F97480F875300185833185823255
:1068E00012043D7881B6FF02800518E6B55207D044
:1068F000F0D5F0C2C322D0F0A3D32222300F0CC2B5
:106900000F1267DE40051277B080031277CF7885CB
:10691000E6C45403E6540F7886E6C45401E6540FE7
:106920007884E6C4540FE6540F7883E6C4540FE627
:10693000540F30080A12685F50051268FB8003127A
:1069400069AB22C2AC127302C2AC12831C12831C4C
:10695000D299C2B674FF1258E875380074421258C2
:10696000E874621258E874151258E8742A1258E84C
:10697000741B1258E874001258E874001258E87436
:10698000001258E874001258E81202D575F010C0D1
:10699000F074001258E8D0F0D5F0F4E5381258E859
:1069A0003099FDC24FD2B612730222222014012266
:1069B0007475787912012F501A206819D268126FF5
:1069C000617518C075190B741A543F4400F51A12FA
:1069D00009C422C2681277CF2033042034332278CE
:1069E00084E6543FF5F0796FE365F0702109E378B0
:1069F0008366701A203516D235126F617518C0750E
:106A0000190B741A543F4400F51A1209C422303489
:106A10002F7884E6543FF5F07971E365F070210931
:106A2000E3788366701A203516D235126F617518B7
:106A3000C075190B741A543F4400F51A1209C42288
:106A4000C23522C2AC120A02600CF5188819120D68
:106A500043120A1A80EFD2AC227E007F849000009D
:106A600075F000E49325F0F5F0A3C3E5829EE5837D
:106A70009F40F0E5F070022200E5F0C0E0E58312EF
:106A800067DDE5821267DDD0E01267DDC2ADC2AC22
:106A9000D216C2A012009420B7F875F0C81282EC8A
:106AA000D5F0FA30B7FD75F0C81282ECD5F0FA12C5
:106AB00073022275F032128304B2B5128304B2B5A8
:106AC000D5F0F32275F06412059120E50430E3015E
:106AD00022C2AFB2B5128304B2B5128304D5F0E777
:106AE000126E8D126AB3126E92126AB3126E8D120A
:106AF0006AB3126E92126AB3126AB3126AB3126A5E
:106B0000B380DD2230083C7400788912013E4033A6
:106B10007F087E007478787912012FCE13CE05E0BD
:106B2000DFF420170E7400789912013E5005EE65CF
:106B30005460108E548E527518C075190485521AFF
:106B40001209C422C2AF75181075190FF51A12096F
:106B5000C4D2AF22223008FC205CF974017889127B
:106B6000013E40F07477787912012FE492E0C0E0A2
:106B70007476787912012FD0E033FE20170E74015D
:106B8000789912013E5005EE655560C88E55EE208D
:106B9000E10630E028026BD030E014A25E725D5056
:106BA000B3C25EC25D126E7174F8126B4480A5D2DE
:106BB0005EC25D126E7174F7126B448097205D0E99
:106BC000D25DC25E126E71D25B74F6126B44808429
:106BD000A226825D40F8D25DC25E126E8574F51207
:106BE0006B44026B54C082C083D083D08222223097
:106BF0004309C2A3C256D2A4C25722D2A3C256C2CC
:106C0000A4C2572220080122300819C0E0C082C067
:106C1000837407120188D083D082D0E04003026CD5
:106C200042026C24201708206033D260205F2ED2ED
:106C30005FD2607518C0751900751A0F1209C40269
:106C40006C5D201708306015C260305F10C25FC2F3
:106C5000607518C0751900751A101209C43008192A
:106C6000C0E0C082C083740F120188D083D082D06C
:106C7000E04003026C97026C79201708206233D23F
:106C80006220612ED261D2627518C0751900751A22
:106C9000511209C4026CB2201708306215C262306A
:106CA0006110C261C2627518C0751900751A52125E
:106CB00009C422C2B675380074031258E8E51E12E2
:106CC00058E8E51F1258E8744E1258E87408125834
:106CD000E874011258E874061258E87848E2F5F0B2
:106CE000E5F01258E808E2F5F0E5F01258E8784AC5
:106CF000E2F5F0E5F01258E808E2F5F0E5F0125898
:106D0000E82442F8E2784CE2547FF5F07844E2C39C
:106D10006001D3E5F092E7F5F0E5F01258E875F080
:106D200000E5F01258E8E5381258E83099FD22C223
:106D3000B6127CD8127C6775380074031258E8E5E7
:106D40001E1258E8E51F1258E8744E1258E8740CE9
:106D50001258E874001258E8740A1258E8C082C049
:106D600083A3A3A3E49375F064A4C0E0E5F01258F4
:106D7000E8D0E01258E8A3A3A3A3E49375F064A4B9
:106D8000C0E0E5F01258E8D0E01258E8D083D08295
:106D9000E4931258E8A3E4931258E8A3A3A3E4935E
:106DA0001258E8A3E4931258E8E58D1258E8E58BF1
:106DB0001258E8E5381258E83099FD22C2B612128E
:106DC000FEC0E075380074031258E8E51E1258E85A
:106DD000E51F1258E8744E1258E874041258E8740B
:106DE000021258E874021258E8E57E1258E8D0F012
:106DF000E5F01258E8E5381258E83099FD22C2B69D
:106E0000121241C0E075380074031258E8E51E12F2
:106E100058E8E51F1258E8744E1258E874041258E6
:106E2000E874021258E874021258E8E57E1258E835
:106E3000D0F0E5F01258E8E5381258E83099FD2214
:106E4000C0F088F0C0F0C2AF7576007850E2F54C23
:106E5000F5F008E2F54DD2AF45F0D0F0A8F0D0F053
:106E60007009B226202604126E7B22D22675760384
:106E700022C2AF754CFF754DFFD2AF757600C209C7
:106E8000C226D2A722126E40D25BD25522C26E0217
:106E9000824CD26E02824C305D1220260F543F4449
:106EA00000F51A7519087518C01209C422C0E0C887
:106EB000C0E0E47868F208F2D0E0F8D0E022C0E068
:106EC000C8C0E0E87869F218E4F2305D08202605D1
:106ED00078687401F2D0E0F8D0E022C0E0C8C0E0E9
:106EE0007868E2601408E2543F4400F51A75190806
:106EF0007518C01209C4126EADD0E0F8D0E022D2ED
:106F0000B2C2B4D293C322D2B2C2B4D29312830417
:106F100020B2ECC29312830430B2E4D29312830401
:106F200012830420B2D9C29312830412830430B2B4
:106F3000CED2B2C2B4D293D322120488C284745483
:106F40001204A2E4120462120475F5F06448255E8E
:106F500033F55EE5F0255FB2E003F55FD9E9D28451
:106F6000227583DD75F0107530038583317532002D
:106F7000C083C0F0120347120860D0F0D0830583AD
:106F8000D5F0E47533FF7534FF757700757800220E
:106F9000E5822400C0E0E58334DDF8D0E0C322C000
:106FA00082C0837401F97480F8753003858331855C
:106FB000823212043D7880B6020CE57824FFF57821
:106FC000E57734FFF577D083D08222126F90C082AC
:106FD000C083F5828883126F9F788076007401F9F0
:106FE0007480F8753003858331858232120392D024
:106FF00083D08222126F90C082C083F5828883C0C2
:1070000082C0837401F97480F875300385833185FB
:10701000823212043D7880B60209D083D082D083B8
:10702000D08222E5782401F57850020577D083D00C
:1070300082788076027401F97480F8753003858354
:1070400031858232120392D083D08222126F901245
:107050006F90C082C083F5828883126F9F7880769C
:10706000017401F97480F8753003858331858232AB
:10707000120392D083D08222126F90C082C083F517
:10708000828883126F9F788076037401F97480F888
:10709000753003858331858232120392D083D0828A
:1070A00022126F90C082C083F58288837401F974C4
:1070B00080F875300385833185823212043D7880F3
:1070C000E6B40102800CB402028007B4030280021D
:1070D0007400D083D08222120488C28474541204B3
:1070E000A2E4120462120475B40205755E01800206
:1070F000D9F3D28422755E007583DD75F00F75308B
:1071000003858331753200C083C0F0120347120437
:10711000B812034779001270D7D0F0D0830583E509
:107120005E7026D5F0D87530038583317532001234
:1071300003471204B812034779A01270D77533FFC2
:107140007534FFE55E7002D322C322E5784577608F
:10715000167866E2F5F008E245F0600BD37867E256
:10716000957818E2957722C3221270A1C2B67538BD
:107170000074031258E8E51E1258E8E51F1258E89B
:1071800074501258E8747D1258E8900000E536609B
:107190000F9003E81460099007D0146003900BB8B7
:1071A0007E7D7F0875F000C0F01270A1B40203D399
:1071B0008001C3D0E033F5F0A3DFEC1258E8DEE243
:1071C000E5381258E83099FD22C28C758A45758CD5
:1071D0005DD28CB20020000132C000C001C0D0C01E
:1071E000E0C0F075D008D25412115B1272E3051D95
:1071F000E51D20E00C20E10930161AE51D541F6042
:1072000056201604E54B6002B2B5D0F0D0E0D0D0E5
:10721000D001D00032205905A226B392A2E51D303C
:10722000E203127F8DE51D541F702FD255C2727874
:10723000AAE2D5E006D271D272743CF2C082C08359
:10724000127E79D083D082E4B54745B54957B563FE
:107250005FB56F60B57F64B54A65E4B54B43B5482B
:107260006CB5456DB54E71B57672E54D454C601DFA
:10727000E54D2401F54D5002054C454C700FC209F7
:10728000205C0A205D07126E7BD25BD25502720130
:10729000D547B8C2097549B4757D00D247D24A8036
:1072A000AA154B80B9D549A6C245C246C247809EA1
:1072B0001563809DD56F9DC2708099157F8098D58C
:1072C0004A987546033016030265BD8081154880D3
:1072D00090D54590D24E808C154E808BD5768BC242
:1072E000A78087E51DA2E330560292A3305902928F
:1072F000A230580292A122C2B6204F02D2B6127317
:10730000023275C800C2ADC2AC75CBFF75CA9875A4
:10731000CDFF75CC98759853C298C299D2ACC2BCB7
:1073200075C8347599062275C800C2ACC2AD75988F
:107330000075CC2B75CDEBD2AD75C8042275C80095
:10734000C2ACC2AD759800E58A242BF5CC540F650C
:107350008C24EBF5CDD2AD75C80422C2A8C2AAC256
:1073600089C28BC2ACC2A9C2AB758F0112059ED275
:1073700016126E92126E71E4F53C7854F2787975BB
:10738000F010F2D5F0FCC25CC25DC25EC25FC261A9
:10739000753EFF7540FF751D04C244C245C246C21A
:1073A00047754901754A00C24AD254757300C23507
:1073B000C218C219D24EC24F754510E4F541F542CC
:1073C000F543F535F537121ED2751E00751F80E4A2
:1073D000F547F550F54FF558F559F53FC223C2244E
:1073E000C225C22B74377859F2785AF2785BF2785A
:1073F0005CF2D21F75460375480178AC7A0576FFBA
:1074000008DAFBC20F7818E47A07F208DAFCC21037
:107410007552FF855254C211C208757F0375631EF1
:10742000756500C267C20DC20EC209C20AC20BC294
:1074300063C26475610075600075F0067842E4F21D
:1074400008D5F0FB7948E4F309F3794AF309F378B6
:107450004CE4F2121470754BFAB2B57533FF753403
:10746000FFD268756E007827740AF2127CB7C2707A
:10747000756F0175721AC201C202C203C204C2054D
:10748000D2A075760075770075780078A974FAF245
:10749000E478B1F278B2F278B3F278AA743CF2C22E
:1074A00074C273C26F757D00127DECC275D276C254
:1074B00077758901758A3E758C5DC2B9D2A9D28C67
:1074C000D2B6127302D2AFD293C2B4D2B2B2B52244
:1074D000C21675510375F0031282ECD5F0FAC2633F
:1074E000C26412369275510375F0031282ECD5F026
:1074F000FAC263C264123531C2AF02000020051324
:1075000020040820020D200102C3221214841278E4
:10751000C2D3221279CBD32275F000C0F012235BC4
:10752000D0F0500343F008E5F022307314204322DA
:1075300078B3E2307106C271600214F224FA500985
:107540002230740E78B3E27009E57C5401700312A6
:1075500000E422C274C273E478B3F222C2AF754B66
:10756000FAB2B5128304B2B5128304B2B5D2A075D3
:1075700081D775D00012735B126BE5126A59126FD6
:1075800061121D45754BFA120C411274FD755103C1
:1075900012380C1238221200F17518807519047512
:1075A0001A801209C4D21730080F120A92126B0403
:1075B000126B551269AC126C04D2B7D2AFC216C2AC
:1075C0001700000020B70912830420B703021D5FD3
:1075D000300832120A9212752AE57A542060117826
:1075E000A9E2D5E00A1277CF12694378A974FAF2BA
:1075F000E57D6002157D30080C126B04126B55128C
:1076000069AC126C04E5656003D5650B127DE5126B
:1076100039061268FC800CD2A3C256C2A1D258D23D
:10762000A4C257E5637003126A43C259D2A1C2587B
:10763000126BEFC263C264D25B785FE2600D24FD1F
:1076400040097575021239F51274FD7860E2600D1B
:1076500024FD40097575031239F51274FDE579545E
:1076600040600620A80312337C12215920510820C3
:107670005005205202801A302F09304606126BE561
:107680000276891245161274FD7827E215E0F27031
:107690000878277414F20275B90275F00074A2120A
:1076A0007731E812776CE912776C1277A32274A213
:1076B000127731E812776CE712776C09D582F812ED
:1076C00077A32274A2127731E812776C74A3127731
:1076D0003112778CF709D582041277A322C296D291
:1076E00097000000C29780E974A2127731E8127700
:1076F0006C1276F52274A312773112778CF9127717
:10770000A32274A27A08C296000000C297335005E3
:10771000D296027717C296D297000000C297DAED90
:10772000D29600D297000000309604C297C322D3AD
:10773000227A08D296D297000000000000000000D4
:1077400000000000000000C296000000C297335005
:1077500005D296027758C296D297000000C297DAF7
:10776000EDD29600D297000000C297227A083350DB
:1077700005D296027778C296D297000000C297DAB7
:10778000EDD29600D297000000C297227A08D296D6
:10779000C29700000000D297C3309601B333DAF0ED
:1077A000C29722C296000000D297000000D2962213
:1077B000788076000876007884E6543FF678007981
:1077C00080C0827582071276AED0821282EC227857
:1077D000027982C0827582051276C3D082227886B1
:1077E000E603C4540775F018A4C0E07884E6C454D6
:1077F0000375F00AA4F5F0E6540F25F0D0F025F05B
:1078000075F03CA4C0F0C0E07883E6C4540775F07E
:107810000AA4F5F0E6540F25F0D0F025F0F5F0D0ED
:10782000E03400C5F022207556206921C0D0C0E0A8
:10783000E8C0E0C0F0E54E7003857270754E08D266
:107840006C12793ED0F0D0E0F8D0E0D0D0C28932CE
:10785000206929C0D0C0E0E8C0E0C0F0E54E700368
:10786000757000754E08A2B2B3926C127A233085FF
:1078700002D203D0F0D0E0F8D0E0D0D0C28B32C238
:10788000A8C289322075C9206926C0D0C0E0E8C0EE
:10789000E0C0F0E54E7003857270754E08C26C1240
:1078A000793E308502D203D0F0D0E0F8D0E0D0D0DD
:1078B000C28B32C2A8C2AAC293C2B4C0E01282EC88
:1078C000D0E0C275C293C2B4C289C28BD2B2D2B365
:1078D000C269754E00857270C203C2B8D288D2A840
:1078E000C2BAD28AD2AA22C275C2A8C2AAC289C208
:1078F0008B22E572141475F00884F5F0C0F0782E30
:10790000E230E002B26A30E102B26A30E202B26A08
:1079100030E302B26A08D5F0E7D0F0E230E002B21C
:107920006B30E102B26B30E202B26B30E302B26B59
:1079300008D5F0E7206A05306B02C322D322E57038
:10794000B57207A26C926A027988B40107A26C92A0
:107950006B027988C3E572149570403275F0048427
:10796000242EF8E205F0D5F006A26C92E38016D53D
:10797000F006A26C92E2800DD5F006A26C92E18036
:1079800004A26C92E0540FF2D57002D26922857283
:1079900070D269227548321278B3305405C254123D
:1079A000027AE54860113069F1E570700A1278E7F3
:1079B0001278F24002C3221278E7D322C2A8C2AAE8
:1079C000C293C2B4C0E01282ECD0E0D275C293C2BE
:1079D000B4C289C28BD2B2D2B3C269754E0075707F
:1079E00000C203C2BAD28AD2AA227548321279BC26
:1079F000305405C25412027AE548600C3069F1E552
:107A00007070051278E7C3221278E7D322C330E002
:107A100001B330E101B330E201B330E301B330E44C
:107A200001B322E57075F00584C0E024ECD0E0409D
:107A300055242EF8E2A26C92E503F2E570700BE299
:107A4000541FB40B40757005803B0570E5F0B4041D
:107A500034E2127A0D502F540FF218E2540FB40F83
:107A600024D3E8942E782EF20404C082F58275F0B7
:107A70000B08E265F0F5F0D582F7D082540F70065E
:107A8000D269757000221279CB220100000000003B
:107A9000000000000A0000000000000000000406D2
:107AA0000000000000000000080E030000000000BD
:107AB000000000010702000000000000000A0608A4
:107AC000010000000000000402040F00000000009C
:107AD000000806090809000000000000010E050F5B
:107AE0000500000000000A0C0A090B03000000005A
:107AF000040E0B00040502000000080E060708042F
:107B0000070100000001050A040D080E75F00A794E
:107B100098770009D5F0FA782EE2FA60400824F24E
:107B20005007EA24F328F87A0DE2540FF26029EAAC
:107B30001475F00AA4248AF5827400347AF58379E6
:107B4000A17E007B0AE493F5F0E2A42E2775F010E5
:107B500084FEA7F0A319DBED08DACEC322D32209F5
:107B60004300A00954009F0966009E0977009D0903
:107B700089009C099B009B09AD009A09BF009909E7
:107B8000D2009809E4009709F700960A0A00950ABE
:107B90001D00940A3000930A4300920A5700910A8C
:107BA0006B00900A7F008F0A93008E0AA7008D0A4F
:107BB000BB008C0AD1008B0AE7008A0AFE00890B01
:107BC0001400880B2B00870B4300860B5C00850B91
:107BD0007500840B8E00830BA700820BC100810B04
:107BE000DB00800BF6007F0C10007E0C2B007D0C60
:107BF00047007C0C64007B0C81007A0C9E00790CA1
:107C0000BB00780CDB00770CFB00760D1B00750DBC
:107C10003B00740D5B00730D7D00720D9F00710DB4
:107C2000C200700DE4006F0E07006E0E2C006D0E8A
:107C300051006C0E76006B0E9B006A0EC100690E3F
:107C4000E900680F1100670F3900660F6100650FCA
:107C50008900640FB300630FDE0062100900611039
:107C6000340060105F005F7F42907B5FE493A3F578
:107C7000F0E493A3C3958BE5F0958D5015A3A3DF96
:107C8000EBE58224FFF582E58334FFF583E493146A
:107C9000800BA3E493BF4205907B5F8010C0E0E5BA
:107CA0008224F9F582E58334FFF583D0E022900049
:107CB0006AE0A28733F02290006B7400F090006AB3
:107CC0007455F090006C74FFF090006E7405F090A5
:107CD000006D7412F0D28122D286A2A4C0D0D2A4A8
:107CE00075F000D5F0FDD5F0FDC28E53890F4389A4
:107CF00010758B00758D00C28FC2AFC2A4D28E20CA
:107D00008603308FFAC28E308F06758BFF758DFF1C
:107D1000D2AFD0D092A422F024FE4005308102C21E
:107D2000812290006EE0D5E0EE7442F0127CD8D251
:107D300081E58B2499E58D34F24014E58B24E1E54F
:107D40008D34F3400EE58B24E0E58D34FC4008745F
:107D5000158006741180027412FE90006DE06E6052
:107D600013EEF0E5795404700B7518C07519008E88
:107D70001A1209C422127CAE603904603690006C7D
:107D8000E020E010D2E0F090006BE070047405F0A9
:107D900022E4F02290006BE0602C14F07028E5796A
:107DA000540270227518C0751900751A141209C48E
:107DB000027DC690006CE030E00DC2E0F090006BF8
:107DC000E070CE743CF02290006BE060F914F0702B
:107DD000F5E579540270EF7518C0751900751A131E
:107DE0001209C480E1127D22127D75229002EB758A
:107DF000F008E4F0A3D5F0FB9002F375F00874FFEF
:107E0000F0A3D5F0FB22C0E0127E59D0E0B3502C95
:107E1000C0E024F8D0E04022C082C083F5F024F313
:107E2000F582E43402F583E0C5F024EBF582E43416
:107E300002F583E5F0F0D083D082D322C0E024F8AD
:107E4000D0E04013C082C08324EBF582E43402F515
:107E500083E4F0D083D082C322C0E024F8D0E04095
:107E600016C082C08324EBF582E43402F583E0D0AF
:107E700083D0826002D322C3229002EB75F008E027
:107E80006003B4FF05A3D5F0F62220E70414F080C8
:107E9000F43072F114F0B480ECE4F080E8B4400700
:107EA0007400127E59803DB441077401127E5980DE
:107EB00033B442077402127E598029B44307740315
:107EC000127E59801FB444077404127E598015C075
:107ED000E024E4D0E04013232455C0E07400347F54
:107EE000C0E022C3740122D380FAE4C322A243B3C8
:107EF00080F2D255A26F80EC80F0A20980E6A20B3E
:107F000080E2A27780DE80DF80E0A20A80D6307037
:107F1000D280D4E577457860CA80CC12714B80C49A
:107F2000A25E725DB380BDA25D822680B7A25DB005
:107F30002680B1A25E80ADC330730920430678B3BA
:107F4000E27001D3809EA26EB38099C3E57F600189
:107F5000D38091809580968099809780958093803A
:107F600091808F808D809180918093809580978083
:107F70009780978099809C80A280A580AA80AE80FF
:107F8000B280B480C180C480CA80C880C61280A27A
:107F9000300819C0E0C082C0837404120188D08305
:107FA000D082D0E04003027FCB027FACE539B40D34
:107FB0000A3021028035D221D3801EB4160678D231
:107FC000E6C38015127E9D6022800EE539B40D0651
:107FD000202103027FEBC221C34009C227A227B39D
:107FE00092A58007D227A227B392A5300819C0E036
:107FF000C082C0837405120188D083D082D0E04053
:1080000003028026028007E53AB40D0A302202807E
:1080100035D222D3801EB4160678D3E6C38015125B
:108020007E9D6022800EE53AB40D06202203028078
:1080300046C222C34009C228A228B392A68007D212
:1080400028A228B392A6300819C0E0C082C0837469
:108050000B120188D083D082D0E0400302808102DD
:108060008062E53BB40D0A302A028035D22AD380E3
:108070001EB4160678D4E6C38015127E9D60228059
:108080000EE53BB40D06202A030280A1C22AC3409C
:1080900009C22CA22CB392808007D22CA22CB392BE
:1080A0008022B20C300C60E57A5410600330431B20
:1080B000E57B54047003204538E57B5401700320B0
:1080C0004611E57B54027003204717C26F755000BC
:1080D000028107E550B401028024755001754F40BC
:1080E000801CE550B402028015755002754FA080C7
:1080F0000DE550B403028006755003754FF0E54F4F
:1081000023F54FA2E0926F22C227A227B392A522A5
:10811000D227A227B392A522B227A227B392A522E3
:10812000F5F00303543FB40258E53964086005E5EF
:1081300039B40D4AE5F089F0C0F0300819C0E0C04C
:1081400082C0837404120188D083D082D0E04003BF
:10815000028165028156D0F0A9F05403B4020D12D9
:10816000810802824AD0F0A9F002824AB4010612C4
:10817000811002824AB4030612811802824A0282E6
:1081800048B40362E53A64086005E53AB40DEFE5EA
:10819000F089F0C0F0300819C0E0C082C0837405D7
:1081A000120188D083D082D0E040030281C40281D2
:1081B000B1D0F0A9F05403B40211C228A228B3929E
:1081C000A602824AD0F0A9F002824AB4010AD2285B
:1081D000A228B392A602824AB40309B228A228B305
:1081E00092A680668062B4045FE53B64086005E5A2
:1081F0003BB40D54E5F089F0C0F0300819C0E0C080
:1082000082C083740B120188D083D082D0E04003F7
:10821000028228028216D0F0A9F05403B4020FC2E1
:108220002CA22CB392808022D0F0A9F0801CB40143
:1082300009D22CA22CB392808010B40309B22CA2D4
:108240002CB3928080048000D322C322C0E0741734
:10825000306E21B53907C227A227B392A5B53A07D8
:10826000C228A228B392A6B53B07C22CA22CB39277
:1082700080D0E022B53907D227A227B392A5B53A1C
:1082800007D228A228B392A6B53B07D22CA22CB3C2
:108290009280D0E022B4010775190F751AE122B45B
:1082A000020775190F751AE222B4030775190F75C5
:1082B0001AE322B4040775190F751AE422B41107E2
:1082C00075190F751AD122B4120775190F751AD2C4
:1082D00022B4130775190F751AD322B41407751930
:1082E0000F751AD42275190F751AD422C28E5389AC
:1082F0000F438910758BD6758D97C28FD28E308FB4
:10830000FDC28E22C28E53890F438910758BEB7587
:108310008DCBC28FD28E308FFDC28E22C28E5389FA
:108320000F438910E58AC4242BF58B758DEBC28F22
:10833000D28E308FFDC28E22543F4400F51A75193B
:108340000A7518C00209C4543F4480F51A75190A09
:108350007518C00209C4543F4400F51A75190C750C
:1083600018C00209C4543F4440F51A75190C751819
:10837000C00209C4543F4480F51A75190C7518C021
:108380000209C4543F44C0F51A75190C7518C0028F
:1083900009C47401127E3C7404127E3C2200000069
:1083A00000000000000000000000000000000000CD
:1083B00000000000000000000000000000000000BD
:1083C000000000000000000000000000000050520B
:1083D000343032207665722E3132382E322E3220F1
:1083E0004864773A482032392D30362D30352032E6
:1083F000323A30372020004352430000000000751D
:00000001FF
:0300000306028072
